:020000040800F2
:10000000301100200101000807380008D12800083D
:1000100005380008350F0008516400080000000092
:100020000000000000000000000000007D49000802
:100030009F1A0008000000006D3D00087D4C00087C
:100040001B010008653B00081B0100081B0100089C
:100050001B0100081B0100081B0100081B01000810
:100060001B0100081B0100081B0100081B01000800
:100070001B0100081B010008591500081B0100089E
:100080001B0100081B0100083D0700081B010008B8
:100090001B0100081B0100081B0100081B010008D0
:1000A000ED4C0008D94D00081B0100081B01000899
:1000B000DD4D0008CD500008295300081B01000841
:1000C0001B0100081B0100081B0100081B010008A0
:1000D0001B010008495F00081B0100081B01000804
:1000E0001B0100081B0100081B010008DFF80CD0F1
:1000F00000F0E6FA004800475D7500083011002066
:100100000648804706480047FEE7FEE7FEE7FEE7B1
:10011000FEE7FEE7FEE7FEE7FEE7FEE79D4C000890
:10012000ED0000082DE9F0410024061B254671F181
:10013000000605DA01240027D0EB070067EB010178
:10014000161E73F1000605DA0027D2EB070201251F
:1001500067EB030300F0D0F986460E4617469C462F
:10016000AC4204D00025D0EB050E65EB010624B1AE
:100170000020D2EB000760EB030C704631463A4694
:100180006346BDE8F08140EA01039B0703D009E024
:1001900008C9121F08C0042AFAD203E011F8013B73
:1001A00000F8013B521EF9D2704780EA010210B5F7
:1001B00002F00043400022D04A001FD0010E01EBA4
:1001C0001261C0F35600C2F3560240F4000042F43C
:1001D0000002A0FB022000047F39140400D0401C60
:1001E00050EA124001D44000491EC2B20C0604EB92
:1001F000D010401C4008802A02D003E0002010BD2F
:1002000020F00100002900DA0020184310BD2DE97C
:10021000FE4F81EA030404F0004421F00041009401
:100220004FF0000B23F0004350EA01045ED052EA85
:1002300003045BD0C3F30A54C1F30A552C44A4F25F
:10024000F3340194A0FB0254C1F3130141F4801173
:10025000C3F3130343F4801301FB024400FB034E7A
:10026000840A970A44EA815447EA8357A4FB076843
:1002700002958D0A05FB07854FEA932C04FB0C546D
:100280002705029D4FEA065847EA1637B5EB0805E1
:100290006EEB070C870E920E47EA811742EA831233
:1002A000A7FB0201B6EB0B0164EB00042B0D43EA44
:1002B0000C335E1844EB1C50DA465146E7FB020152
:1002C000C5F313044FEA0B3343EA14534FEA0432E5
:1002D000019C43EA0603A4F10C040294009CCDE9BE
:1002E00000B400F09FF903B0BDE8F08F0020014694
:1002F000F9E72DE9F04D81EA030404F0004B21F009
:10030000004514464FF0000A23F0004150EA050270
:1003100020D054EA01021DD0C5F30A570246C5F3A6
:100320001303C1F31300C1F30A5640F4801543F4DC
:100330008013A7EB0608101BD64608F2FD3873EBB6
:10034000050002D308F1010801E092185B41B8F101
:10035000000F03DA00200146BDE8F08D00204FF4C5
:100360008011064684460EE0171B73EB050705D384
:10037000121B63EB050306434CEA010C49084FEAE4
:10038000300092185B4150EA0107EDD152EA0300B8
:1003900012D082EA040083EA0501084305D0101B4D
:1003A000AB4106D20122002306E000224FF00043B9
:1003B00002E06FF0010253101AEB06004CEB0851FB
:1003C00010EB0A0041EB0B01BDE8F04D00F01BB94A
:1003D00070B521F0004303430CD0C1F30A5500244B
:1003E000D5EB040564EB0403D617AD1AB34102DB69
:1003F0000020014670BD201841EB025170BDC10FB5
:1004000080EAE0700844CA079623002100F0CDB8C6
:1004100096230022114600F0C8B80EB5C10F80EA3D
:10042000E0700844CA07002140F233438DE80E0013
:100430000A460B4600F0F6F803B000BD0EB540F2D8
:10044000334102910021CDE900110A460B4600F02C
:10045000E9F803B000BD00F0004220F00040C10DFB
:10046000C0F3160040F400007F2901DA0020704735
:10047000962903DCC1F19601C84001E09639884015
:10048000002AF4D04042704770B5C1F30A5201F01F
:1004900000450024C1F3130140F2FF3341F4801101
:1004A0009A4201DA002070BD40F233439A42A2F230
:1004B000334203DC524200F05FF800E090402C43EE
:1004C000F1D0404270BDC1F30A5210B5C1F313011F
:1004D00040F2FF3341F480119A4201DA002010BD4E
:1004E00040F233439A42A2F2334203DC524200F01C
:1004F00043F810BD904010BD2DE9F05F0546002087
:1005000092469B4688460646814640241BE0284684
:1005100041464746224600F02FF853465A46C01A35
:10052000914110D311461846224600F016F82D1AB4
:1005300067EB01084F4622460120002100F00DF82C
:1005400017EB00094E41201EA4F10104DFDC4846F0
:1005500031462A464346BDE8F09F202A04DB203A74
:1005600000FA02F1002070479140C2F1200320FA06
:1005700003F3194390407047202A04DB203A21FA04
:1005800002F00021704721FA02F3D040C2F12002AC
:1005900091400843194670470029A8BF7047401C86
:1005A000490008BF20F00100704710B4B0FA80FC89
:1005B00000FA0CF050EA010404BF10BC704749B1C6
:1005C000CCF1200421FA04F411FA0CF118BF012136
:1005D00021430843A3EB0C01CB1D4FEA00614FEA16
:1005E000102042BF002010BC704700EBC3501044E5
:1005F0000029A4BF10BC7047401C490008BF20F070
:10060000010010BC704710B5141E73F1000408DA25
:10061000401C41F1000192185B411A4301D120F0C6
:10062000010010BD2DE9F04D92469B4611B1B1FA83
:1006300081F202E0B0FA80F220329046FFF78DFF9F
:1006400004460F4640EA0A0041EA0B0153465A4667
:10065000084313D0114653EA010019D0C8F14002F3
:100660005046FFF789FF05460E465046594642461A
:10067000FFF773FF084305D0012004E02046394608
:10068000BDE8F08D0020054346EAE0762C43374371
:100690000A986305E40AA0EB08000022FD0A44EA78
:1006A00047540A3002D500200146E9E70105101938
:1006B0006941DDE9084500196941BDE8F04DA2E74F
:1006C000064C074D06E0E06840F0010394E807009F
:1006D00098471034AC42F6D3FFF70CFD2C99000874
:1006E0004C99000870B58C1810F8015B15F00703E1
:1006F00001D110F8013B2A1106D110F8012B03E0BB
:1007000010F8016B01F8016B5B1EF9D12B0705D4C2
:100710000023521E0DD401F8013BFAE710F8013B0B
:10072000CB1A921C03E013F8015B01F8015B521E27
:10073000F9D5A142D8D3002070BD000070B54C4C53
:100740004FF490652946204600F015FA002864D041
:100750002946204600F0A2F846490888401C088037
:100760000121204600F0E6FA434942F21072B1F846
:100770005000904202D2401CA1F8500007F0D6F879
:100780003E4DB5F91410B5F9120005F093FF3C4C3D
:10079000A5F856002080A16820468847A088A5F8C3
:1007A000580003F099F807F0BDF9364E364C307812
:1007B000082833D045F6AC30606042F6EF60A060A8
:1007C00042F2C400E0603148008A2080208E6080C0
:1007D000A16B2D488847208E69882D4C08444FF620
:1007E000FF7101EA80006887207A4FF0000540071A
:1007F0001DD501F0E3FA274949F6A24008802648B2
:1008000040F21A62C188491C89B2C180914204D366
:10081000A16821F00401A160C58070BD41F2130000
:1008200060604FF48060A06040F61B50CAE73078EB
:100830000A2818D2DFE800F0170613050A050D177D
:100840001113EAE7BDE8704006F0DEB808F050F991
:1008500005E0BDE8704002F089BD06F05BFCBDE834
:10086000704007F0B7BA00F0FDFB84F8B65070BDD9
:1008700000240140240700204801002064000020DB
:10088000440700201B070020E4000020F80100209E
:10089000A4020020442C0140640900206FEA1121C9
:1008A000016070470029816802D041F0010101E038
:1008B00021F00101816070470029816802D041F474
:1008C000807101E021F48071816070472DE9F04171
:1008D000824E92B0304600F00BF90BA800F039FAC6
:1008E00001214FF4C06003F0D5FA00248DF83140A7
:1008F0004FF46020CDE90D044FF4A0204FF009081B
:100900000B9001278DF83C808DF830700BA9304694
:1009100000F080F9724D8DF831408DF830708DF80F
:100920003C700BA9284600F075F901231A460F21E7
:10093000304600F0C0F9022201231146304600F093
:10094000BAF9012303220021304600F0B4F9012353
:1009500004221946304600F0AEF9012305220B218E
:10096000304600F0A8F9012306220421304600F0A9
:10097000A2F9012307220821304600F09CF9012347
:1009800008220321304600F096F9012309220A21AA
:10099000304600F090F90121304600F084F9012141
:1009A000284600F080F901231A460521304600F060
:1009B00055F901231A460621284600F04FF9002177
:1009C000304600F0CBF84FF4E041284600F0C6F87E
:1009D0000121304600F0B8F80121284600F0B4F8B3
:1009E0000121304600F0A6F80121284600F0A2F8C7
:1009F0000121304600F09EF90121284600F09AF9C5
:100A000040F61451374804F066FF12208DF840007C
:100A100002208DF841008DF842408DF8437010A8F7
:100A200002F01EFF01224FF49061304600F0E8F81A
:100A300001213046FFF740FF01213046FFF732FF2A
:100A400001212846FFF72EFF304600F06EF93046B0
:100A500000F09FF80028FAD1304600F075F93046D2
:100A600000F082F80028FAD1284600F05EF9284606
:100A700000F08FF80028FAD1284600F065F92846E2
:100A800000F072F80028FAD10121084603F0DEF9DF
:100A9000154D284600F09CFD684600F044FE0F48C6
:100AA00001A94C300090114881E811018020CDE966
:100AB00004404000069080000790202008904FF4EA
:100AC0004050CDE909046946284600F00FFE012197
:100AD000284600F071FD12B0BDE8F081002401400D
:100AE00000280140002C014008000240B402002010
:100AF0000D4910B5884202D1012144150AE00B4985
:100B0000884202D10121041504E0094988420AD132
:100B10000121CC03204603F0C9F92046BDE810406E
:100B2000002103F0C3B910BD00240140002801409A
:100B3000003C01400029816802D041F4801101E0AD
:100B400021F48011816070470029816802D041F44E
:100B5000004101E021F4004181607047826822F485
:100B6000E0420A43826070470146002089684907D5
:100B700000D50120704710B50246002054680B0ACA
:100B8000C9B20C401168194202D0002C00D00120DB
:100B900010BD014600208968090700D50120704773
:100BA00038B501211C2003F075F9FF20ADF80000D5
:100BB00000248DF8034003258DF8025069460D4846
:100BC00001F0F6FA0120ADF800008DF803408DF831
:100BD00002506946084801F0EBFA2320ADF8000006
:100BE0008DF803408DF802506946044801F0E0FAA0
:100BF00038BD000000080140000C01400010014019
:100C0000002A4268C9B201D00A4300E08A43426028
:100C10007047000010B542680E4B0C791A400B6803
:100C200042EA04221343436083680B4A1340D1E92C
:100C3000024222434C7943EA44031A438260C26A67
:100C4000097C22F47002491EC9B242EA0151C16214
:100C500010BD0000FFFEF0FFFDF7F1FF70B50724A7
:100C600009290AD9C568A1F10A0606EB4606B4406F
:100C7000A543B3401D43C56007E0056901EB41068C
:100C8000B440A543B3401D430561836BC3F30154D6
:100C9000121B921C02EB82041F22A2409343A1402C
:100CA0000B43836370BD826B491E22F4401242EAFB
:100CB00001518163704770B5072409290AD9C568B5
:100CC000A1F10A0606EB4606B440A543B3401D4316
:100CD000C56007E0056901EB4106B440A543B34098
:100CE0001D4305611F23072A09D2446B521E02EBE4
:100CF000820293409C4391400C43446370BD0D2A93
:100D000009D2046BD21F02EB820293409C439140B4
:100D10000C43046370BDC46A0D3A02EB8202934037
:100D20009C4391400C43C46270BD816841F008014E
:100D3000816070470029816802D041F4A00101E080
:100D400021F4A00181607047816841F00401816055
:100D5000704700210160017141718160C160012112
:100D60000174704770B51E4C214694F83800B1F8F4
:100D7000425006281ED9B4F84A10B4F84C00A1EB32
:100D8000000202F10902122A04D8FFF757FB0022E1
:100D9000144B0AE0884204D2FFF750FB0022124BAA
:100DA00003E0FFF74BFB0022104BFFF730FAFFF791
:100DB0008AFB09E005D12846FFF740FB0C4A0D4BA2
:100DC000F3E70D4951F82000C5EB45116063B0EB26
:100DD000410F03D9C5EB45104000606370BD0000B2
:100DE0005004002000003440000033400000354033
:100DF0006766666666E64B40DC8F000810B50C4CF3
:100E00002078400713D5FFF7ADFF0A49A08E088070
:100E100008483038018821F010010180001F018846
:100E200041F010010180207820F00400207010BDF6
:100E30005004002040040040F0B4184816494FF414
:100E40009677436C08468A68046815485FEAC25C76
:100E500042F00806007822F008054FEA047415D520
:100E6000002C08DB120714D408B1082811D1BB42AA
:100E70000FDA8E6007E012070BD508B1082808D1F9
:100E8000BB4206DA8D60F0BC05F046BF002CF2DAFA
:100E9000E8E7F0BC70470000A402002048010020F1
:100EA0001B07002070B506464089204B204C4FF4AC
:100EB0008071002580B362887AB1012A0CD1E18863
:100EC000491C89B2E1803289914205D36580E58071
:100ED000FF2801D0401E708170BD7088228890422A
:100EE00001D9012200E00022184601F0EAF97088D9
:100EF000B18801442088401C80B220808142EBD818
:100F00002580A088401C80B2A080F1888842E3D36D
:100F100001206080A58070BDFFE70022184601F027
:100F2000D0F9A580E58025806580F4E7000C0140BC
:100F3000C0050020FEE70000FCB505464FF6FF7631
:100F400000200C46ADF8006048F205078DF804005B
:100F500020E000BF15F8010B8DF8040001A9084638
:100F600002F0E1F8BDF800009DF8041080EA0120CD
:100F7000ADF800005FF00000BDF800100A0402D5D3
:100F800087EA410101E006EA4101401CADF800108A
:100F90000828F1DB641EDDD26946084602F0ADF890
:100FA000BDF80000FCBD00000246002004E000BFC8
:100FB00012F8013B1844C0B2491EF9D27047000034
:100FC00070B5144A85B01088002413490194009428
:100FD000039420460494138807E00D8B009E35444B
:100FE0000095CD8B019E3544019515889D42F4D026
:100FF000401CC0B28028EED30098411107484180C0
:10100000848001984111064881830183818205B063
:1010100070BD000024070020A4020020DA05002093
:10102000C804002030B50E4902880A800C4A438863
:10103000083A13800B1F808818802024151F2C80ED
:101040000020401C80B27328FBD341F211100880AD
:1010500044F64800108047F2480018802C8030BDCC
:10106000202C0140114944F648000880091D46F62D
:1010700048000880091D41F2111008800B48001F2C
:10108000018841F02001018009480021A0F8641086
:10109000A0F86210A0F86010A0F85E10A0F85C1034
:1010A000A0F85A100348418181827047182C0140F2
:1010B000A4020020640000202DE9F04F524B534859
:1010C0000022D97A90F800C080292CF001067DD347
:1010D0001C684F4B01F01F0153F821104D4B0C427F
:1010E000196802D041F0200101E021F02001994669
:1010F0001960484BDFF820B1DFF820A193F8465083
:10110000474B9BF80040B3F90430022C69D1B9F881
:101110000840C4F3C007C4F30024A74261D03D4C8B
:101120002C3C94F80280B8F1000F09D0374FB8F189
:10113000010FB7F902700DD0B8F1020F56D120E0BF
:101140000A0553D58A0651D40122A2702CF004025C
:1011500002704BE00E0549D48E0647D55FEA4C7607
:1011600044D4A7BB4380002B09DD4CF0050202707C
:101170000222A2702B4AB2F84420028236E0A2700A
:1011800034E0B0F806C0BCF1000F01D1002B17DC31
:1011900090F80CC0AC4513D107F26667BB420FDC78
:1011A000214FBF895FEA477C0AD45FEA877C07D476
:1011B0005FEA417C04D55FEA816C01D5FF0715D059
:1011C00006704280AAF80020428101E017E00DE09D
:1011D000426182610282A27089F80F208BF80020A0
:1011E00004E006704280AAF800204281C3800573A3
:1011F000480960F3CB21C9F80010BDE8F08F0670F4
:1012000042804281F9E70000E00500204809002003
:101210003C940008A40200201B07002024010020A9
:10122000DA05002048010020580A00202DE9F04787
:1012300096B000240C940D940E940F9472B69048BE
:10124000816941F400718161816941F4806181614A
:101250004FF4004002F0F0FD8A4D00212846FFF7D0
:101260002BFB00212846FFF71DFB874E002130464F
:10127000FFF718FB854F0021384600F09DF901204B
:101280004FF47041401C8842FCD32846FFF730FCE5
:10129000B1463046FFF72CFC384600F099F94FF480
:1012A0006020CDE912048DF8454001204FF004087C
:1012B0008DF8440010948DF8508010A92846FFF74F
:1012C000A9FC01231A4605212846FFF7F4FC012357
:1012D000022206212846FFF7EEFC01230322072104
:1012E0002846FFF7E8FC012304220F212846FFF7D8
:1012F000E2FC384600F06CF9684600F014FA6148E8
:10130000634E4C300090CDF80C80CDE90164802014
:10131000CDE904404000069080000790202008900E
:101320004FF44050CDE909046946384600F0DEF933
:1013300001212846FFF7C0FA0121384600F03CF9A8
:1013400001212846FFF7AEFA47F23051159415985F
:10135000401C15908842FAD301212846FFF7EAFC89
:10136000ADF82C40A04640F2DC5A4FF4007420E067
:101370005046CDF854801599491C15918142FAD3F5
:1013800030880D9908440D9070880E9908440E908D
:10139000B0880F9908440F90F0880C9908440C907D
:1013A00001212846FFF7C6FCBDF82C00401CADF813
:1013B0002C00BDF82C00A042DAD30D98354A40F33A
:1013C000CF1633480A3006830E9941F3CF14448375
:1013D0000F9941F3CF1383830C9941F3CF1CA0F8ED
:1013E00004C0ACF5C05C40F2C371ACF59B7C8C458D
:1013F0000ED2A6F5C856363E8E4209D2A4F5C85480
:10140000363C8C4204D2A3F5C853363B8B4203D3FF
:10141000D18841F48041D180D188490407D41E4944
:10142000028B21F85C2F428B4A80808B88800021C0
:101430002846FFF741FA0021384600F0BDF80021A8
:101440002846FFF72FFA00214C464846FFF72AFAB4
:101450000220C102401C8842FCD32846FFF748FB0B
:101460002046FFF745FB384600F0B2F8FFF72EFAAA
:101470000A493C20087062B616B0BDE8F08700004B
:1014800000100240002401400028014008000240F2
:1014900026050020580A0020B80C0020180700205C
:1014A000F0B52B4B40F22D4643F6FB255C6C294BE7
:1014B000B4F5FA5F13DDB4F5FA4F10DC41F6AD1761
:1014C000A4F5FA54674306EBA7364FF4B5777C438F
:1014D00005EBA41475106410C3E9045401E0C3E9DA
:1014E00004654FF46A74D4604FF48344401A546125
:1014F00010609168884202DA4942884200DC11603B
:1015000010684FF483414843117E0841916A0144B9
:101510009162506A814200DD9062916A106A814254
:1015200001DB084600E09062986111684FF46A732D
:101530005943137C194118410144B2F91C008842F7
:1015400004DBB2F91A00884200DC08B2F0BD0000EA
:10155000480100202801002010B54FF40054204617
:1015600000F0ACF8002813D00A49087840F00800D1
:101570000870204600F014F80021074800F01CF81D
:101580000648C17E012903D10021C17601210177DE
:1015900010BD00007A060020440002405C0B0020D1
:1015A000C10002D50249086070470249486070478F
:1015B00004040240000002400029016802D041F00A
:1015C000010102E04FF6FE72114001607047000019
:1015D00001684FF6FE721140016000210160416018
:1015E0008160C1603149314A0839904203D148686D
:1015F00040F00F0006E02D4A1432904204D14868B2
:1016000040F0F00048607047284A2832904203D1E9
:10161000486840F47060F5E7244A3C32904203D1B8
:10162000486840F47040EDE7204A5032904203D1C0
:10163000486840F47020E5E71C4A6432904203D1C8
:10164000486840F47000DDE7184A7832904203D1D0
:10165000486840F07060D5E7154A111F904203D1E9
:10166000086840F00F0006E0114A1432904204D19D
:10167000086840F0F000086070470D4A2832904238
:1016800003D1086840F47060F5E7094A3C329042A3
:1016900003D1086840F47040EDE7054A50329042AB
:1016A000EAD1086840F47020E5E700000800024035
:1016B00008040240406880B27047000001460020E4
:1016C000CA0001D5034A00E0034A12680A4200D06A
:1016D000012070470004024000000240002A026816
:1016E00001D00A4300E08A430260704730B50368C6
:1016F00047F6F07293430C6A8A682243D1E90445A5
:101700002C4322438C692243CC6922434C6A2243F6
:101710008C6A22431A430260CA6842600A68826087
:101720004968C16030BD0021016041608160C160D5
:10173000016141618161C161016241628162704701
:1017400010B5114C8CB000212046FFF735FF204624
:10175000FFF73EFF0D4800900D480021CDE9010143
:101760006420CDE903018020CDE9050107910891AE
:1017700009910A9169462046FFF7B8FF01212046EA
:10178000FFF71AFF0CB010BD5800024004380140AA
:10179000B407002010B501218CB0084602F056FBBA
:1017A0001E4C00212046FFF707FF2046FFF710FFE1
:1017B0001B4800901B48019000211020CDE9020138
:1017C0008020CDE9041006910791089109910A91B2
:1017D00069462046FFF78AFF012202212046FFF7D3
:1017E0007DFF01218DF82F1004208DF82D008DF83C
:1017F0002E100E208DF82C000BA802F031F80F20CF
:101800008DF82C000BA802F02BF801212046FFF7E1
:10181000D3FEFFF795FF0CB010BD0000440002405E
:10182000043801405007002030B540F6AA21204A74
:10183000C184838B1488E31A9BB20F2B10D31288B8
:101840008283037E002253B11A4BB3F90A30062B70
:1018500005DB194B1B78022B03D0002B00D18284AF
:1018600030BD164B40F68B255B6CA3F22D14AC42B9
:101870000FD2428B521C92B24283642AF0D364226C
:101880004283B0F924208A4201DA02EB21118184DB
:1018900030BD41F29414A342FADBB0F92430002B9E
:1018A00002DDA3EB211100E000218184428330BDE1
:1018B00024070020640000201B07002048010020AE
:1018C00010B50446B0F9020043F69911484381135C
:1018D000E06840F26662504301EBA030E060B4F98A
:1018E000001043F6991251438A13216940F266634E
:1018F000594302EBA131216104F07CFE6061A188B3
:1019000040F6AB2208444010A0F515415539E0627D
:10191000914205D9A0F5F851FF39521C91421DD2D0
:1019200049F25451884202DDA0F5204002E0A0F5C2
:10193000F850FF38206300EB400040F34F00208553
:10194000B4F924104A42904201DA104602E088427B
:1019500000DD0846E083228461848AE0A0F5FE422F
:10196000FF3A41F255518A4214D8A2F6AA202063C8
:1019700000EB400040F34F002085B4F92420514291
:10198000E183884201DA084602E0904200DD104619
:10199000404250E0A0F5D442AA3A8A4215D2A2F6BB
:1019A000AA20206300EB400040F34F012185B4F9E9
:1019B00024004242E2832084914201DA104602E090
:1019C000814200DC0846608453E0A0F5AA42543A04
:1019D00041F256539A4215D2A2F6AB20206300EB97
:1019E000400040F34F002085B4F924104A42904251
:1019F00001DA104602E0884200DD08464042E083FA
:101A0000218419E0A0F5804241F254539A4215D244
:101A1000A2F6AA20206300EB400040F34F0121858D
:101A2000B4F92400E0834242914201DA104602E018
:101A3000814200DC0846208462841AE0A0F5285226
:101A4000AB3A8A4215D2A2F6AA20206300EB4000EE
:101A500040F34F012185B4F92400E08342422284FF
:101A6000914201DA104602E0814200DC0846404221
:101A7000A9E7B4F91E00A0EB40208013E080B4F980
:101A80002000A0EB402080132081B4F92200A0EBBD
:101A900040208013608110BD01210176704770479E
:101AA0001548164A4FF480410078042821D002F1ED
:101AB0003C03D08A9B88C01A00B22F2801DD001198
:101AC00008E0002801DD002007E00D4B984201DA14
:101AD000184602E0402800DD40209389184400B2F7
:101AE000884203DC40F26661884200DA0846908151
:101AF00070479181704700001B070020C804002038
:101B0000C0FEFFFF38B54B484B4902880B889A1A34
:101B100092B20F2A71D30988484C01804FF0FF011F
:101B2000E2884FF47A7355044FF4967002D516226A
:101B3000009103E0950403D515220091014670E061
:101B4000D50402D514220091F8E7150502D5132219
:101B50000091F3E7550502D512220091EEE79505B5
:101B600002D511220091E9E7D50502D51022009196
:101B7000E4E7150602D50F220091DFE7550602D5EE
:101B80000E220091DAE7950602D50D220091D5E7E5
:101B9000D50602D50C220091D0E7150702D50B22FD
:101BA0000091CBE7550702D50A220091C6E79507B9
:101BB00002D509220091C1E7D20702D00822009184
:101BC000BCE72289550702D507220091B6E79507A1
:101BD00002D506220091B1E7D20702D0052200917A
:101BE000ACE7A27AD20702D004220091A6E7A2892C
:101BF000D40603D503220091A0E719E0140702D50B
:101C0000022200919AE7540703D4940701D4D20723
:101C100002D00122009191E70020034602460146CE
:101C2000009002F057FFBDE838400248FFF73AB98C
:101C300038BD00004C0A002024070020580A00206C
:101C4000F0B55948594982880B889A1A92B29C2A51
:101C500064D30988818056490A880146002A0B7896
:101C600043F0020156D11646524A1C071568024637
:101C7000127822F0020274D54F4C0746E4887F7830
:101C80005FEA845C02D547F0010701E027F0010715
:101C90004770A704477802D547F0020701E027F014
:101CA00002074770670401D4E70703D0477847F07D
:101CB00008074770640603D5447844F0040404E040
:101CC0001C0603D4447824F004044470EC0450D47B
:101CD000354C9A07247824F0100423D4324D4278EE
:101CE0002F7A2D78012A45F0100514D0022A16D03B
:101CF0002D4C042AA47804F1010C0CF0FF0C13D035
:101D0000072A25D0032A23D0052A21D0062A1FD04E
:101D100021F0100142E0B90702E00570F0BD39077B
:101D20000029FADB0470F0BDFA0601D41A060AD5C0
:101D30000170022C04D280F802C0BCF1020FF2D371
:101D400041F080012AE021F0100101708670F0BDA1
:101D5000877A7F06F7D5032C04D8017080F802C07B
:101D6000F0BD0FE05107D8D51906D6D443F0800155
:101D700014E002704178CB0701D18907F0D522F039
:101D800010010BE0E9040BD49907E9D4818AC82932
:101D900002D2491C8182E3E743F00A010170DFE7C8
:101DA00002708682DCE70000FC0600202407002089
:101DB00026070020A4020020580A0020094944F602
:101DC00048000880091D46F648000880091D41F6B4
:101DD000CC4008800348001F018841F020010180A9
:101DE00070470000182C0140084946F6680008803A
:101DF000091D0880091D41F2555008800348001F45
:101E0000018841F02001018070470000182C01403A
:101E100010B5C28800210AB1032206E002890AB186
:101E2000022202E0428912B10122027000E0017038
:101E300004784FF4804344F6206244B1012C06D06C
:101E4000022C07D0032C01D14180818010BD43803A
:101E5000828010BD41F23331418040F6B731F4E762
:101E600030B5B1F86A5000231A240D22854202DCF5
:101E7000B1F9680030BD4D88854202DBB1F9000040
:101E800030BD01EB82056D88854201DD144601E01D
:101E900013DA134604EB03024FEA52029A42F0D1DE
:101EA00001EB830231F8231054889288521A001BE8
:101EB000424301EB622000B230BD31F9220030BD57
:101EC000054920B1086940F0800008617047034867
:101ED000486003484860704700200240230167457E
:101EE000AB89EFCD06494FF47A70CA68D20705D0A6
:101EF000401E0004000CF8D1FF20704700207047FE
:101F0000002002400E4A0320A2F1500182F83E0058
:101F1000002048810B490886C862C8830884488429
:101F200090620948816CB1F5206F01DBA3219162B9
:101F3000807A002802D0906A404290627047000088
:101F400064000020300500204801002004490020E2
:101F500048810881C862886202498862704700002F
:101F600064000020C4080020F0B53B4988894A89F4
:101F7000801A80B20F2866D388894881CA89374879
:101F80000B3A272A26D28A7822BB8268364B42F443
:101F900080728260324A354C354D12785607314A8C
:101FA0000AD4344E36881680334A12881A80334A4F
:101FB00012882280324A09E0324E36881680324A30
:101FC00012881A80314A12882280314A12882A8067
:101FD00001228A702F4B304D19469A7F0968802A5A
:101FE00032D302F01F0255F8222011422CD0826811
:101FF00022F48012184E8260123614461215B778F9
:10200000521C62F38617254AB77093F816C01778EA
:10201000BCF1800F27F0020608D30CF01F0C55F816
:102020002CC011EA0C0F01D147F0020616701A7E7F
:10203000802A0DD302F01F0255F82220114207D149
:1020400044F400218160F0BD826842F48012D1E73F
:1020500024F40021F6E7000018070020A402002065
:1020600048010020C0040020C2040020C404002055
:10207000C6040020B0040020B2040020B4040020F4
:10208000B6040020B8040020BA040020BC040020DC
:10209000BE040020E00500203C940008C804002095
:1020A00070B5204881890289891A89B20F292FD3F6
:1020B000818901811C4B1D4819465D7A06681C4CBC
:1020C000096846F00402802D07D305F01F0554F877
:1020D0002550294201D126F0040202609A7B802A11
:1020E00017D302F01F0254F82220114211D10268C6
:1020F00022F002020260DA7A802A0ED302F01F0276
:1021000054F82220114208D1016821F00801016031
:1021100070BD026842F00202ECE7016841F008017C
:10212000F5E7000018070020E0050020A4020020C9
:102130003C940008F0B51D4C1B4A4FF0010C94F87C
:102140003B5094F80AE0144692F83C3094F838403A
:102150002B43651CEEB2154D95F83D700025BEF180
:10216000FF0F0AD0BEF1000F06D18B4213D155707C
:102170000C2C01D282F83860F0BD834202D182F883
:1021800001C0F5E78B42F7D15570B80709E000BFF1
:1021900082F83850F0BD8342FCD1F84382F801C088
:1021A00080070028F4D0F0BD500400204801002032
:1021B000F0B5CA78002502F00F03D20601D58A785F
:1021C00013430A784FF00F0E12F0FF0F4FF0010289
:1021D0001CD004680F8802FA05F63740B74211D1C7
:1021E0004FEA850C0EFA0CF724EA070703FA0CF401
:1021F0003C43CF78282F02D0482F02D002E046611E
:1022000000E006616D1C082DE4D304600C88FF2CEF
:102210001ED944685FF0000606F1080702FA07F5C8
:102220000F882F40AF420FD14FEA860C0EFA0CF701
:10223000BC4303FA0CF73C43CF78282F00D145610B
:10224000CF78482F00D10561761C082EE4D3446076
:10225000F0BD0000F0B5144C002801DAE36900E09D
:102260006368420D120185B2C0F301579540C0F377
:102270000346032F05D0C2020AD50322B24093437E
:1022800007E023F07062636823F07063636002E02C
:10229000AB4343F0706201B12A43002801DAE261E6
:1022A000F0BD6260F0BD0000000001400246002069
:1022B00092680A4200D00120704741617047016175
:1022C00070470AB101617047416170470F4A104B76
:1022D00092F838105B5C834201D1012004E00D4B81
:1022E0005B5C834203D1002082F83A0070470A4BBE
:1022F0005B5C834201D18120F6E7084B595C814247
:1023000001D18020F0E70320EEE700004801002023
:10231000F498000806990008FA9800080C9900083B
:102320000A4810B501784FF000024C0708494FF0F9
:10233000FF0389684FEA017105D5002901DA82722D
:1023400010BD837210BD0029FBDBF8E748010020B7
:10235000A4020020F0B5194E194C0022E31CA6F18E
:10236000060CB75CA518ED78FF5C0D430F43BD422A
:102370001FD01CF80270FF5C0F43BD4219D01546F8
:102380000023A618F6780E43C6545B1C1CF80220E6
:10239000DBB2062BF5D3C17881700179C1700021C1
:1023A0004218491C15711CF80550C9B20629F7D30B
:1023B000F0BD521CD2B2032AD3D3F0BDCE8F000899
:1023C0005004002010B502460021064B06205C1880
:1023D0006478944200D10846491CC9B20629F6D354
:1023E00010BD000048010020214810B590F867108A
:1023F00000222048012936D11F49898899BB1F49ED
:102400001E4B4C6C40F6B831B3F86E308C4227DD71
:102410001B49097821BB90F82711491CC9B280F8E3
:102420002711C8291CD380F827210146D0F82C4158
:1024300091F82811A34203DD052908D2491C01E0C7
:1024400041B1491E80F82811C9B2052902D30121E2
:1024500080F82611191B074C2C3C6162C0F82C3106
:10246000B3F5FA6F03D280F8262180F8282110BD39
:10247000B80C0020A4020020DA050020480100204A
:102480001B0700204FF4C042C260002181620E226F
:10249000028241F262024261082202834FF46042EA
:1024A000428381834FF07842C0E9082140F6C4118D
:1024B00001807047B0F90010B0F90220891A41601C
:1024C0004269037E4A431A41836A13448362426A23
:1024D000934200DD8262836A026A934200DA82627A
:1024E000C268836A4A43017C0A410B41D118B0F9A2
:1024F0001C208A4201DA10467047B0F91A0088425F
:10250000FADC08B27047000010B514481449B0F85E
:102510008C200B889A1A92B2B2F5437F1DD9098894
:10252000A0F88C10B0F88A1020F8581F00224286BC
:102530000C480D4CC2888280C180C3898381248964
:10254000891AA4B2C4818160E11A0161074A818AB3
:10255000C182928A8282511A816110BD4801002095
:1025600024070020800C002030050020640000209B
:1025700009480A49B0F8AA200B889A1A92B241F683
:1025800084639A4206D3098820F8AA1F4188818073
:1025900000214180704700004801002024070020EE
:1025A0000D480178C90702D00C49098801E04FF6AF
:1025B000FA71C1650949012010390880074824389B
:1025C000018841F00101018004481838018821F098
:1025D00018010180704700004801002024040040D9
:1025E0000A49D1F8902012B1521EC1F8902031F85A
:1025F0008A2F521C21F81A294A6A521C4A628A8F71
:10260000521C8A8701F8380C7047000048010020EE
:102610001CB52D4890F83B3090F83C20934252D0A6
:1026200000248DF8044053408DF800309DF80030B0
:102630000122012B08D09DF80030022B09D09DF813
:102640000030042B0AD00DE01F498DF804204431DE
:1026500008E01D498DF80420463103E01A498DF841
:10266000042048319DF80420012A2CD190F83D30F7
:102670009DF80040154AA34217D090F83E309DF8CF
:102680000040234208D0B0F84C30A0F84A300B8804
:102690001488E31AA0F84C3090F838302BB1B0F819
:1026A00040301488E31AA0F8423012880A80A0F85B
:1026B000402010F83E1F9DF80020114300F801193A
:1026C0009DF8001001701CBD50040020240700205C
:1026D00070B5344D40212846FFF7E8FD8400802185
:1026E0002846FFF7E3FD44EA4004A9152846FFF712
:1026F000DDFD0443E1B22C4C94F870508D4250D073
:102700004D4084F87010012D03D0022D01D0042D0E
:1027100047D194F87400A84384F8740094F87320A7
:10272000AA420FD084F8735094F8722001238B4092
:102730001A4207D11A4384F8722094F87110491C88
:1027400084F8711094F87110042928D330B101284D
:1027500011D002280FD004280DD012E01348C188F0
:1027600021F04001C1802078002184F83B1020F046
:102770006000207005E0217841F02001217084F88C
:102780003B000B4994F83B0091F82720904204D07D
:1027900081F8270007492020087000F00DF884F820
:1027A0004C5070BD0010014048010020580A002024
:1027B000B80C00201807002070B50D4D40212846A8
:1027C000FFF774FD840080212846FFF76FFD44EA7F
:1027D0004004A9152846FFF769FD04430548072171
:1027E00000F8704F0171002141708170C17070BD9F
:1027F000001001404801002070B5344890F83A10AC
:10280000CA43920761D001F0030280F8392090F8A2
:102810003D305B061B0E80F83D30012A01D0812A35
:1028200002D15B1C80F83D300278D2074DD0DBB27C
:1028300003F00102C3F34004A24246D1B0F84E4077
:102840000025641CA0F84E40204CA0F8505090F891
:102850003E60A47AB24202D080F83E200DE0A60786
:10286000B6EB837F02D080F83F5006E090F83F300F
:10287000642B02D25B1C80F83F3090F84030642B10
:102880000CD25B1CDBB280F84030022B06D204F085
:102890000103934202D1022280F84020012901D095
:1028A000002912D190F83820C16D00EB82029161AD
:1028B0000163D0E906121144D0E908231A441144F7
:1028C000826A1144C26A1144416370BD480100200C
:1028D000FEE700002DE9F04F00BF00209E4E9F4A0A
:1028E000A6F51271A6F5BE79A6F1440B06F1440EC9
:1028F000804601F5E074A1F1780301F5457A1D5C8D
:1029000015F0C00706D0402F51D0C02F77D0802FB0
:1029100076D004E115F01F0504D0154440F080077F
:102920002F7201E082F80880012826D0022824D0E6
:10293000032822D0042820D008281ED010281CD01C
:10294000874D55F820C0DCF8005054F820703D4009
:10295000CCF80050824D55F820C0DCF8005056F8F5
:1029600020703D43CCF800501D5CAD0659F8205056
:102970002F6813D53AF810C03EE051F820502F6868
:1029800054F820C007EA0C072F6051F820502F6838
:1029900056F820C047EA0C072F60E5E7DFF8B8C11A
:1029A0000CF1F00C5CF820C007EA0C077EE015F093
:1029B0001F0504D0154440F080072F7201E082F813
:1029C000088001281DD002281BD0032819D0042814
:1029D00017D0082815D0102813D0614D55F8205075
:1029E0002F6854F820C007EA0C072F605C4D55F89B
:1029F00020502F685BF820C047EA0C0756E00BE038
:102A000056E051F820502F6854F820C007EA0C0710
:102A10002F6051F82050ECE715F01F0505D0154444
:102A200040F0800785F8217001E082F821800128BC
:102A300025D0022823D0032821D004281FD008281D
:102A40001DD010281BD0464D55F820C0DCF8005092
:102A500054F820703D40CCF80050414D55F820C04E
:102A6000DCF800505EF820703D43CCF800501D5C4F
:102A7000AD0615D53A4D3AF81070CC3514E051F842
:102A800020502F6854F820C007EA0C072F6051F837
:102A900020502F685EF820C047EA0C072F60E6E759
:102AA0002D4D3AF81070E03D55F820502F6036E07B
:102AB00015F01F0505D0154440F0800785F82170FA
:102AC00001E082F82180012830D002282ED003288E
:102AD0002CD004282AD0082828D0102826D0204D11
:102AE00055F820C0DCF8005054F820703D40CCF878
:102AF00000501B4D55F820C0DCF80050164F8837A9
:102B000057F820703D43CCF800501D5CAD06B1D4A1
:102B1000114F3AF81050E03F57F820703D60401CCC
:102B2000C0B21128FFF4EBAEBDE8F08F51F8205091
:102B30002F6854F820C007EA0C072F6051F8205086
:102B40002F68DFF814C00CF1880C5CF820C047EA4D
:102B50000C072F60D9E70000C8960008E0050020A8
:102B6000C49400084FF40771C1824FF45861018387
:102B700040F6145181837047F0B5C48AB0F9006003
:102B80008681B0F90250C581B0F9043002270021D6
:102B900001220382AB4204DBB54202DDC7804281E1
:102BA0000CE0B34204DBAE4202DDC78041811CE091
:102BB0009D4205DBB34203DDC2804781018115E000
:102BC000B54204DB9E4202DDC280418105E0AE4297
:102BD00005DB9D4203DDC1804281078106E09E4204
:102BE00004DBAB4202DDC18047810281C388458995
:102BF00000EB430700EB4505BB89AE899B1B0FFA31
:102C000083FEA0F812E00689AB8900EB460CBCF805
:102C10000CC0A3EB0C038382B0F91830B7F90CC0D9
:102C2000A3EB0C0CB4EB4C0F04DA80F82010A3F1EA
:102C3000A10113E0A64503DD80F82010B9890BE05F
:102C400026B1012E04D0022E10D004E0062100E0AF
:102C5000052180F82010A989091B6D31418309B233
:102C6000B1F5586F04DB5B1E438304E00421F0E7F9
:102C7000002900DC4283418B8183F0BD0B49002297
:102C800088760A62CA614A62094A32F9103002EB58
:102C900040028B62B2F90220CA62064A32F8100082
:102CA0000882A1F86000A1F862007047F8010020D6
:102CB0001E990008129900082DE9F05FFD48FE49B1
:102CC00082880B889A1A92B20F2A44D30988FB4A49
:102CD0008180814611880124F948FA4E002579B394
:102CE000491E1180C573F84A85620168B2F9022055
:102CF0004F0742F6AA2318D4F78847F40057F78005
:102D0000F14E3678B60709D5866826F080068660CB
:102D1000A0F87C5080F87E5080F87F50CE0404D418
:102D200080F8F040C0F8EC5003E080F8F0504E0717
:102D300007D49A4205DB80F8F440A0F8F25004E092
:102D400010E080F8F4504E0703D49A4201DBC90723
:102D500003D080F81151BDE8F09F80F81141A0F830
:102D60001251F8E78046B0F8181143F698208142D6
:102D700002D2491CA8F8181101F0C2FED34FDFF8A7
:102D800034B397F85000ABF11C0B10B1FEF794F977
:102D900005E09BF8001021F001018BF80010FFF70F
:102DA00023FB00F0D7F9CA4841F268024FF40061F2
:102DB000406C904201DBC74A04E0B0F57A6F02DA5A
:102DC000C44A121D116097F85110DFF8F4A2C24BEB
:102DD000C24FC907AAF12C0A3AD0997B802933D374
:102DE00098F8002092072FD498F80F208AF8062030
:102DF000B54A514692F800C02CF0020C82F800C08F
:102E0000ABF80250CBF814509BF800C02CF0010C2A
:102E10008BF800C0B279520611D44A89B2F5FA7F14
:102E200003D2521CAAF80A2012E040F63C729042EB
:102E300001DD002013E108208AF803400FE1CD7086
:102E40000020AAF80A500AE18AF80350AAF80A50AA
:102E5000D8F80800010501D5082000E19B4991F848
:102E60003FE05FEACE7149D09B4B98F80F208AF87B
:102E700006205B7A4146802B4CD30B785B0735D418
:102E8000F3889B0405D500BF20F02000C8F8080097
:102E900034E0ABF80250CBF814509BF800C08E4BD6
:102EA0002CF0010C8BF800C040F020008860D87D29
:102EB00080280AD300F07F0C1B684FF0004020FAF6
:102EC0000CF0034201D10C7100E00D710879C007CC
:102ED00002D15FEA8E7005D50320032A01D08AF85B
:102EE0000940BCE00020C8F82850B8E020F02000DD
:102EF000C8F80800F08820F40050F08098F8260107
:102F0000444601280BD0714890F8630048B1FDF7A2
:102F100093FF0FE00A6842F004020A60B4E7092058
:102F20009DE0A068C10502D520F0080001E040F056
:102F30000800A06094F846304FF48041E3B143F6B6
:102F40009912012B1FD0881E022B2FD03B78C3F380
:102F50008103012B2FD0022B2DD0A4F8141160482F
:102F600090F85E0004281ED0A4F84410574890F84A
:102F70007000012822D031E043F21E50A4F8140161
:102F800043F2333014E0387842F6CC43C0F381008A
:102F9000012806D0022804D043F2EB10A4F8140153
:102FA00001E0A4F81431A4F84420DFE7A4F81401E8
:102FB000A4F84400DAE7A4F81401D0E73878C0F3A5
:102FC000810242F26660012A0FD0022A10D041F637
:102FD000E12200BFA4F81421A4F844009BF80020CB
:102FE000D20708D0BBF8022007E0A4F81401F3E7E9
:102FF0004FF40052EEE734488288A9F8122010B24C
:10300000B4F944205043C0F38F325046AAF812203E
:103010008A4200D9418233490978C90605D5428AD6
:1030200041F233318A4200D241822189C1F3C00288
:10303000C1F300218A4205D1428A40F6CC418A423E
:1030400000D94182B17AC90700D04582BAF812008E
:10305000A06200287FF7EDAE23480570022099F8A2
:103060001A1099B9022841D080B119490B789C06F1
:1030700008D5B479640605D51A4C2478E40964F3BC
:1030800086130B70F18821F40A61F1801049496CB4
:103090004E290ADBF1880B0607D521F08001F1806B
:1030A00009490B7823F002030B7089F81A0088F89D
:1030B0000F0050E6640900202407002026070020A6
:1030C000A4020020580A0020DA050020B80C0020D5
:1030D00048010020100C0140E0050020C804002039
:1030E00064000020FC06002038070020398F0029EA
:1030F000BBD143F698213987B7E770B500230C8818
:1031000063F30F02012505FA03F6344206D0C3F13A
:103110000F0605FA06F1114361F30F025B1C102B39
:10312000F1DB028070BD70B500230C7863F30702F9
:10313000012505FA03F6344206D0C3F1070605FA65
:1031400006F1114361F307025B1C082BF1DB0270EF
:1031500070BD0000F0B51F4890F866301E48012B86
:10316000816821F4006232D11C4BDE8874062ED4B3
:103170001B4D0F054FF00004B5F902501ED4194A3B
:10318000526C642A11DC40F6386295420DDAB204C2
:103190000BD4027852070ED4B0F8D42040F6B835DC
:1031A000AA4203D2521CA0F8D420F0BD41F4006121
:1031B00081605C81F0BDA0F8D440F0BD41F2CD014A
:1031C0008D42FADD997AC907F7D18260F3E7826010
:1031D000F0BD0000B80C0020A4020020580A002016
:1031E000DA05002048010020F0B5364D364F044680
:1031F00095F83B0097F83B1023780843EE1C627863
:10320000834205D1E0781146FEF794FF207908E06B
:1032100094F802C084450CD1E1781046FEF78AFF8D
:10322000E07905F82F0F2878805D6870287BE877B3
:10323000F0BD82421DD161461846FEF77BFF95F82E
:103240004E1095F83B00814207D1B97A09B1A179B6
:1032500000E0617985F82F101EE06978012901D01E
:10326000A17922E0617927E0297841F004012970F1
:1032700012E0E1788142DBD119466046FEF75AFF41
:1032800095F84E1095F83B0081420AD1B97A09B100
:10329000617ADFE7217ADDE715F82F1F895D697014
:1032A000C5E76978012906D0617A85F82F10B97AC7
:1032B0000029F1D1D8E7217A85F82F10B97A0029B1
:1032C000EAD0D1E750040020480100200B480178E3
:1032D00021F0020100F8381B002100F8181941778D
:1032E000817733218185418508214184012100F8BE
:1032F0001F1C034880F8391070470000500400205C
:10330000480100200D4900B50B4851F8012F40F845
:10331000032F89888180084801210930FFF71AF8B6
:10332000054802211330FFF715F8034804211D302A
:103330005DF804EBFFF70EB85004002048010020B0
:10334000094944F648000880091D46F648000880EF
:10335000091D41F2111008800348001F018841F047
:103360002001018070470000182C01402DE9F04732
:10337000664C674B0025A0780126654A1033052866
:103380007ED2DFE800F00313113E1100108820F018
:10339000010010801D805F480580001F0580001F10
:1033A0000580FFF7CDFFA670BDE8F087594941F2CF
:1033B00044401C390880574945F658002439088094
:1033C000091D47F2580008805249202028390880FA
:1033D0000020401CC0B27328FBD3FFF7B1FF4C495B
:1033E00084F85C502C3147F69060088048481430CF
:1033F00006801D80108840F0010010800220A0701F
:10340000D2E700215FF0010004EB410204EB40032E
:10341000B2F85020B3F850309A4200D20146401C16
:10342000C0B20628F0D33C48405C84F83900FFF76E
:103430004DFF1D2000F0F3F900F076F8374E3848C4
:103440004FF4807996F83B10012904D002291BD053
:10345000042930D047E040218046FEF727FF87004F
:1034600080214046FEF722FF47EA40074946404692
:10347000FEF71CFF074347F0010084F83B0000E023
:103480003DE0224809302CE040218046FEF70EFF47
:10349000870080214046FEF709FF47EA400749467A
:1034A0004046FEF703FF074347F0020084F83B0065
:1034B0001648133015E040218046FEF7F7FE8700DE
:1034C00080214046FEF7F2FE47EA40074946404663
:1034D000FEF7ECFE074347F0040084F83B000B487E
:1034E0001D3002F071FF94F82F0086F838001D207F
:1034F00000F0ABF90420A0700A48057054E710886A
:1035000020F0010010801D80A5704DE750040020C0
:10351000000800403C2C0140D48F000848010020E6
:10352000001001401B0700202DE9F041344C14F835
:103530002F0F344DE07240212846FEF7B7FE86007B
:1035400080212846FEF7B2FE46EA4006AF1539460E
:103550002846FEF7ABFE0643207BF1B22F3C8142AA
:1035600015D084F83C0040212846FEF79FFE8600D7
:1035700080212846FEF79AFE46EA4006394628464C
:10358000FEF794FE064384F83B60FFF741F81E4DBA
:1035900095F83B00012827D0022828D0042829D0FC
:1035A000174894F83B102730085C04F8300F14F8E3
:1035B0000109FEF707FF04F82F09A87A00B10120DE
:1035C000607001F035FB94F84E0094F83B1088428F
:1035D00006D094F83800062802D2401C84F838003F
:1035E00084F84E10BDE8F0810548093004E0044835
:1035F000133001E002481D30BDE8F041FFF7F4BD93
:103600005004002000100140480100202DE9F04145
:10361000524991F87200AA287ED191F8730055287A
:103620007AD14F4C00200A5C2254401CC0B274284E
:10363000F9D34C4E2069C6F80100A08AA6F805000F
:10364000D4F81600F060D4F81A003061D4F81E00E7
:103650001234706102F05EFE4349608A888102F094
:1036600073FE207D123CC007307802D040F0040089
:1036700001E020F004003D4930704FF480403C4DA3
:10368000886114F8280F85F82000608B6880A08B73
:10369000A880E08BE880208C2881608C354F688181
:1036A00094F8240087F8D20014F8011C304686F8FC
:1036B0003B100026C0F89460FFF724FE2E48A18E30
:1036C0000183E18E4183218F818394F84210283C4D
:1036D000012908D0022901D0032909D0297821F035
:1036E0000C01083107E0297821F00C01091D02E0E6
:1036F000297841F00C01297094F86E20012162B103
:10370000012A01D0022A0BD087F8461094F86430C1
:103710001A4A4BB1518108E014E087F84660F5E79A
:10372000022287F84620F1E7568194F870100129AB
:103730000AD094F86D1051B101290BD04FF480518B
:10374000A0F87610BDE8F08144F21C71F8E74FF460
:103750000051F5E741F25551F2E7000000FC000886
:10376000B80C00204801002064000020500C00200C
:10377000C8040020A402002030050020580A0020C0
:103780007CB50121082000F085FB4FF48070ADF876
:10379000040010248DF8074001208DF8060001A9CF
:1037A0001548FEF705FD0121092000F073FB0121FA
:1037B0001248FEF74FFD0820ADF8000004208DF8F8
:1037C00003000F4E03258DF8025069463046FEF780
:1037D000EFFC08213046FEF770FDADF800408DF893
:1037E00003408DF8025069463046FEF7E1FC102197
:1037F0003046FEF762FD7CBD00140140000230003F
:10380000000C0140FEE7704700F01F0201219140CB
:103810004009800000F1E020C0F88011704700F0FE
:103820001F02012191404009800000F1E020C0F812
:103830008011704700F01F02012191404009800073
:1038400000F1E020C0F80011704700F01F020121D4
:1038500091404009800000F1E020C0F8001170475D
:1038600070B50F23C47801780122F4B1144C246898
:10387000457804F4E064C4F5E064240AC4F1040665
:10388000E3408478B5401C402C4301F1E021230142
:1038900081F80034007800F01F018A404009800060
:1038A00000F1E020C0F8002170BD01F01F0082404F
:1038B0004809800000F1E020C0F8802170BD0000C0
:1038C0000CED00E00249084302490860704700001F
:1038D0000000FA050CED00E02DE9F05F00261D2048
:1038E000FFF792FF6C4CDFF8B4B1A4F1B000A77EF3
:1038F00090F83810DFF8A8E1DFF8A8A100258F4282
:103900007ED0E776A176626A036B5A434FEA12498A
:103910009BF80820120702D51EF8012000E00A4695
:1039200094F812C0BCF1010F09D004EB4206B6F9BD
:1039300002C0C4F828C0B6F90460E6620CE043F6A1
:10394000FF7CC4E90A5C90F83DC05FEACC7C01D002
:1039500012B102E0052A00D1012600EB47074FF023
:10396000804CBF893F04B7FBF3F3E361476BBCFBBB
:10397000F7F7276294F813C0BCF1000F06D0BCF132
:10398000010F05D03B4403EBD3735B10636201E08E
:103990003B466762DFF810C14FF6FF7707EA8307FF
:1039A000ACF808709AF8007090F80A8090F83DC062
:1039B000082F08F003070CF0030C05D067450BD166
:1039C000B8F1000F05D008E0674505D0B8F1000F49
:1039D00003D05B42636200E06562C6B1636A002B9C
:1039E00003D006DD228D05E00AE0304B33F81220CB
:1039F00000E0A28DA4F86020227822F0200222703C
:103A00009AF80020042A07D0082A05D012E0B4F85A
:103A1000603003EB0902EDE780F8405065629BF8E7
:103A20000800000701D51EF80110204830F81100E9
:103A3000A4F860001E49606A09883E314843B4F822
:103A4000601001EB204006B21D20FFF7F3FE606A14
:103A5000002807D021784FEA81600ADD002804DAC7
:103A6000A08D09E0B4F8600006E0E06AB04208DB2F
:103A70000CE0002802DA208D208208E0A06AB04223
:103A800004DD208241F02000207000E026822575B0
:103A900065752586BDE8F09FF8010020A40200208E
:103AA000009900081B070020300A00201299000826
:103AB0002404004043184FF48042934210DD9042AA
:103AC00002DD104600210BE0914202DD002011468C
:103AD00006E08003B0FBF3F000B2C0F5804109B20C
:103AE00041EA00407047F0B54FF46A730022C360AA
:103AF0000E24826204824FF48345082645610683C2
:103B000043F6FF774283878340F2492E4FEA873C92
:103B1000C0F808E0C0E9082CCB608A620C824D61D5
:103B20000E834A838F83B4208860C1E9082CF0BDDE
:103B3000002181620949C1600E2101824FF6BF5107
:103B40004161082101834FF44041418343F6FF71F5
:103B5000818309070162024941627047638A01005B
:103B600000C0FF0F064941F6A260088005480168C1
:103B7000054A01F4E06111430160BFF34F8FFEE796
:103B8000442C01400CED00E00400FA0538B5012199
:103B90000D2000F07FF94FF4E060ADF8000018242C
:103BA0008DF8034003258DF8025069460D48FEF755
:103BB000FFFA4FF46040ADF800008DF803400A4C66
:103BC0008DF8025069462046FEF7F2FAA014ADF8CF
:103BD000000048208DF8030069462046FEF7E8FA09
:103BE00038BD000000080140000C01402DE9F04103
:103BF0000121CE028CB0304600F04CF9DFF868812C
:103C0000404601F08DFC08A801F0B6FE4FF4586064
:103C1000ADF824000024ADF820402020ADF82200AB
:103C20000125ADF826408DF8285008A9404601F03E
:103C300055FE0021404601F0A8FE4FF6FF714046B8
:103C400001F0ADFE01220021404601F039FE0121C4
:103C5000404601F021FC04A801F039FCADF81060E9
:103C6000A802ADF81200ADF81440A220ADF816007D
:103C7000ADF81840ADF81A40ADF81C4004A9404614
:103C800001F014FC6027ADF80070ADF80440ADF809
:103C90000840ADF80C40ADF80240ADF80640ADF874
:103CA0000A40ADF80E406946404601F0F9FC69460D
:103CB000404601F03BFD6946404601F081FDADF80C
:103CC000045040F61450ADF80070ADF80600ADF8A1
:103CD0000840ADF80C40ADF80250ADF80A40ADF820
:103CE0000E406946404601F0AFFD0121404601F01B
:103CF000F7FB0821404601F013FD3146404601F034
:103D000055FD0821404601F099FD3146404601F03D
:103D1000CDFD7021404601F0D6FD18208DF82C0015
:103D20008DF82D408DF82E408DF82F500BA8FFF701
:103D300097FD0D480C30018841F0800101800A4850
:103D40001430018841F001010180001F048001212D
:103D5000404601F0CFFB8DF828500121404601F08C
:103D6000D3FB0CB0BDE8F081002C0140704740F25D
:103D700013414160082181608621C1604FF4804178
:103D800001614942416100210162C16270470162E3
:103D90007047000010B501884288891A09B2018372
:103DA000B1F5005F02DBA1F5804104E011F5005F91
:103DB00002DC01F580410183B0F9182041685143CC
:103DC000C1618368846A5343C2681B12624303EB78
:103DD0002222036A1A44114402628A134262416930
:103DE0008A4203DB01698A4200DC11468A1AC0E973
:103DF0000A21028E4FF40373594302EBA13202866B
:103E00000B4A1278082A04D10A4A936F03EBA131B6
:103E10009167B0F93010B1F5804F02DDA1F5804116
:103E200003E0002902DA01F58041018610BD00009F
:103E30001B0700206C0A0020034A516821F440410E
:103E4000014351607047000000100240044A0029FD
:103E5000516901D0014300E0814351617047000086
:103E600000100240044A0029D16901D0014300E05A
:103E70008143D1617047000000100240044A0029CC
:103E8000116901D0014300E08143116170470000D6
:103E900000100240044A0029916901D0014300E06A
:103EA000814391617047000000100240044A0029DC
:103EB000D16801D0014300E08143D1607047000028
:103EC0000010024030B524494A6812F00C03234A1E
:103ED00003D0042B01D0082B26D002604A680F23A0
:103EE0001F4C03EA1212A35C0268DA4042604B687E
:103EF000072505EA1323E35C22FA03F383604B688A
:103F000005EAD323E35CDA40C2604B68032403F480
:103F1000404104EA933303EB9161114B1B1F595C41
:103F2000B2FBF1F1016130BD4A680E4B1A404B689B
:103F3000140103F4803303D5C2F38342113202E04B
:103F4000022404EB924213B14B689B0301D5064B4C
:103F500000E0024B5A43C0E70010024000127A0012
:103F60000400002000003C0800093D002DE9F0415C
:103F7000274CA61540212046FEF798F985008021A0
:103F80002046FEF793F945EA400531462046FEF704
:103F90008DF90543EDB240212046FEF787F98700F1
:103FA00080212046FEF782F947EA40073146204645
:103FB000FEF77CF90743F8B2A842DBD14021204646
:103FC000FEF774F9870080212046FEF76FF947EA73
:103FD000400731462046FEF769F90743F8B2A84288
:103FE000C8D140212046FEF761F987008021204694
:103FF000FEF75CF947EA400731462046FEF756F9DE
:104000000743F8B2A842B5D12846BDE8F0810000C8
:104010000010014010B50268416802FB02F301FB89
:1040200001330D4CA34211D91B0E0E3B0B4C9BB21E
:1040300012B234F8133009B25A43594342F38F3263
:1040400041F38F31C0E90221012102E0C0E90221E0
:104050000021017410BD0000E10BBF0E748C00083C
:104060002DE9F05FF948FA4902880B889A1A92B252
:104070000F2A7DD309880180F64802468189D288BB
:104080004B0703D48B0701D4CB0702D042F4007254
:1040900001E022F40072C2808246080702D4504632
:1040A000C90604D5BAF8061041F0010102E0C18842
:1040B00021F00101AAF80610E648FDF7A9FEDFF895
:1040C00098B3BBF93A10B1F5804F03DA491CABF84D
:1040D0003A1003E04FF48040ABF83A00DF4E41F66F
:1040E000CC40DF4CB16C814203DDA06820F01000B1
:1040F000A060DC4ADC4D4FF00008108830B1401E53
:10410000108084F80F8085F800802BE0BAF8060054
:1041100043041BD4BAF80C20D30617D4120715D4C5
:10412000020613D4820611D402050FD4420603D529
:10413000CE4A1278120609D5420707D4C20505D423
:10414000020703D4820401D4C0060BD5C84884F802
:104150000F80C84A85F80080A0F81E80A2F8008071
:1041600080F82A80E08FC44ADFF810E350B100E005
:10417000FAE0401EE087107820F00200107084F80A
:104180000F800AE0107840F00200107028780128B3
:1041900005D19EF80000062801D185F80080287816
:1041A000DFF8DCC2DFF8DC9201270A2877D2DFE8EB
:1041B00000F0FDDB05DBFCFBDB76FAF9DFF8A0A203
:1041C000A648AAF12C0A40F62826BAF81610491C6F
:1041D0008BB2AAF81630416C40F6CC40B14202DAFC
:1041E000AAF8168013E0DBF80C6086420FDBB2F908
:1041F000042043F69916B24209DBB3F5FA7F06D3E1
:1042000099F800301BB9AAF8168089F80070DFF819
:1042100078E2BEF8002072B19AF804305B1CDBB281
:104220008AF80430022B06D38AF80480BCF80020F8
:10423000521CACF80020E27B092A18D0022A7CD05C
:10424000A4F830814FF44050C9F87C00C9F87800D8
:10425000B4F840004E46C8B141F288324046AAF850
:104260001680914221DA3178012919D01DE0774872
:104270004430FEF707F9FDF745FE7848416CCAF86F
:10428000281041F27C51CAF81810B0E2B08A20869A
:10429000F06A7063B06A3063A4F8407036E002E2FE
:1042A0003070ACF80000AEF80000784940F63A22D1
:1042B00091F8681001290DD0C4F8D80084F8EA00FC
:1042C000CAF82000B4F9301001F21D50904217D8FE
:1042D000102316E094F8281101B96D48C4F8D800ED
:1042E00084F8EA70B4F9301001F21D509042B4F82D
:1042F000D80000B201D8102300E02023102202E0F1
:1043000020231022002000F0F1FB20865F48614945
:104310004FF4927390F868000128504815D0406C13
:1043200040F2DC52904203DAB6F90A209A4215DBD9
:10433000B4F84020521C92B200E020E040F6C413D2
:10434000A4F840209A4209D210E0426C40F2DC50BE
:10435000824209DAB6F90A00984205DA85F8008047
:1043600084F8EA80A1F81A80BDE8F09FDBF80C2001
:10437000002AF9DC42F6E0629042EFDAF4E7B4F8A2
:10438000302140F6B8339A4207D2304E1C3E367880
:10439000F60702D1521CA4F8302196B240F2DC524A
:1043A000964204E012E1F0E037E132E13AE102D86E
:1043B00042F6CC4303E0A4F8303143F26663C9F817
:1043C0007C30CAF828108AF80870334AA4F8408074
:1043D00084F8EA80537F5646EBB1D07F174690B3FE
:1043E000208DB4F9301000B20A23052200F07EFBC4
:1043F000208687F81F8087F81D8000BFB4F916015A
:10440000B4F91411884277DA204991F84D10D9B1E6
:1044100000F1020089E01D4D95F86820012A08D1BD
:10442000DBF80C2040F23333DA4202DC94F8262128
:1044300022B194F84600022830D033E0A323B4F927
:1044400030101A4654E05CE063E00000640900208C
:1044500024070020580A00203005002048010020D1
:10446000A4020020280700201B070020FC060020D3
:10447000F40800201E000020DA0500201C070020A0
:10448000220000206400002020000020B80C002042
:1044900034F3FFFFD8090020800C002095F86D0050
:1044A000022813D008B2FA4901F0FAFCA4F8E4009B
:1044B000A16A00B2814200DA084600B2B08295F8E3
:1044C0004D1039B1B4F93010362310E008B2F0497C
:1044D000B031E9E7EF4944F2506240F24713496CCA
:1044E00091420ADD95F8681039B1B4F9301005220F
:1044F00000F0FCFA208681E70DE0B4F93010362296
:10450000F6E740F26660208684F80F8085F8008028
:1045100074E7083009E00BDD7179491CC9B271718B
:10452000022907D386F80580401EA4F8160101E091
:10453000A4F81611D9E91E12914209DAD64A92F866
:104540004D2012B101F102010DE001F108010AE074
:104550000CDD727902F10102D2B27271022A07D324
:1045600086F80580491EC9F8781001E0C9F878205E
:10457000B4F930004FF48041884201DD2186F3E632
:104580000028FCDAA4F83080EEE6C448D4F8DC1049
:10459000814202D2491CC4F8DC10E17B082903D116
:1045A000D4F8DC1081420DD385F80080A068C105E5
:1045B00002D520F0080001E040F00800C4F8DC80DB
:1045C000A060D1E6BDE8F05F02F0BABCE07B09284C
:1045D00004D0A4F8308084F80F8043E1B04DE8693E
:1045E000401CE86102280ADD288D012301B2288BD6
:1045F000052200B200F07AFAC5F81C80A862A9482A
:10460000298D0180B6F844104180FDF753FF2086C4
:10461000AAE6BDE8F05F04F0EFB9A34800780928E6
:104620007ED0A1E694F8280170B141F31100C4F8DE
:10463000D88083039D4AC9F82C00801093628103BF
:10464000C9F828009A4881629548A0F81680716CD4
:1046500041F2883081420ADA99F80010012906D126
:10466000944889F80080ACF80080A0F80080924956
:10467000924B0888401C82B291480A80C82A04D311
:1046800090F800C0BCF1010F1AD0B2F57A7F04D3C4
:1046900090F800C0BCF1020F12D0B2F5FA6F02D34D
:1046A0000278032A0CD0E07BDFF818B2801E0828BD
:1046B00071D2DFE800F0119EDAEC0470659153E6E8
:1046C00080F80080A1F80080BAF8061021F400619B
:1046D000AAF806101F70E6E7FDF722FE30784006C4
:1046E00011D59BF8020004280DD0706C82280ADADC
:1046F000B07A96F83D1000F0030001F00301884203
:1047000001D001F0CDFD287806288AD086F83F80B8
:10471000B06C664A40F311018B03C9F82C1000E01D
:10472000A0E0891093626248C9F828108903816269
:10473000FDF7E8FB5A480772B4F81401A4F8160113
:10474000706CA4F88280B0F5437F06DD4FF48040A2
:10475000A4F8800079E0287006E64FF48041A4F8C0
:104760008010A16821F48061A16040F28A21884212
:1047700004DA3078400601D402F0CEFAA0686CE08A
:10478000706CB0F5437F07DA9EF80010062903D05D
:104790008EF80080A0E0A6E04B48017821F04001AF
:1047A0000170FDF7AFFB43F6FE70A4F81601FDF7AC
:1047B000B7FD464810F8341F21F0010101703C4953
:1047C000C4F8DC80C1F828803849C1F82880082165
:1047D0002970C0F84480C7E53248FDF753FEFDF765
:1047E00091FB2F48716C816241F27C5181610920FB
:1047F000B1E79AF80600C006AED4706CB0F57A7FC7
:1048000030DDFDF78DFD3078400611D59BF80200B4
:1048100004280DD0706C82280ADAB07A96F83D1020
:1048200000F0030001F00301884201D001F038FDDF
:1048300086F83F80B6F84800208601B24FF48040E9
:10484000814200DD2086FDF75DFBA06840F48060BA
:10485000A06096F838100529BDD140F01000A06086
:10486000022078E785F800807EE5706CB0F5437F24
:1048700003DA9EF8001006298AD1BAF8061021F052
:104880002001AAF80610FDF74BFD042063E71FE0A6
:10489000668E000848010020B80C0020C0D401003A
:1048A00078020020A809002060020020C40800202F
:1048B0009408002020000020160000201400002092
:1048C00015000020500400202A0700206C0A002058
:1048D0009EF80000062801D02F7045E50549092003
:1048E0000870052037E78BF802808EF8008089F881
:1048F0005E8047E66002002030B585B001210420CB
:10490000FFF7C8FA4FF40040ADF8100048208DF8CA
:10491000130004A91848FDF74BFC01210846FFF7D6
:10492000A1FA40F68C20ADF8040003240020ADF875
:104930000040ADF80200ADF806004FF08045694632
:10494000284600F0CBFF1C208DF80C008DF80D40A0
:104950008DF80E4001208DF80F0003A8FEF780FFB0
:1049600001221146284600F093FE0121284600F05E
:10497000C1FD05B030BD00000008014070470000D7
:104980002DE9F041304CE07800285AD120780028F9
:1049900057D0401E10F0FF00207052D14FF4967097
:1049A000208272B6294F45F2AA50A7F87200002063
:1049B000FDF786FA264D13202860FDF793FAA8BB71
:1049C0003420E86002202861224E6E61286940F0A0
:1049D00040002861FDF786FA40BB00211E4A0846C8
:1049E0005FEA255312F800C0BCF1FF0F00D001218F
:1049F000401C80B29842F5D3C1B9C4E90676392685
:104A00000127A06910F8011B10F8012BA061E069D3
:104A100001EB022102886A612F6120F8021BE0612C
:104A2000FDF760FA10B9761EB6B2EAD20120FDF7A2
:104A300047FA62B601F088FC0848816821F4804199
:104A40008160BDE8F081000018070020B80C00204C
:104A50000020024000FC000800FC0008A402002026
:104A60001948016841F010010160016821F003015B
:104A70000160016841F00201016014484168416031
:104A800041684160416841F480614160416821F4BE
:104A90007C11416041680E4A11434160016841F058
:104AA0008071016001688901FCD5416821F0030132
:104AB0004160416841F0020141604168C1F38101F8
:104AC0000229FAD170470000002002400010024085
:104AD0000000280830B5044C039D6080A180E2806E
:104AE0002381658130BD00004C0A00200A448242C7
:104AF00001DA10B27047C91A8142FBDD08B2704773
:104B00002DE9F0434348DFF81081DFF81091C17FB1
:104B1000457A046801260023414A424880292BD364
:104B200001F01F0158F821100C420146096802D01B
:104B300041F4805101E021F480510160CF0417D489
:104B40008F0415D5977AFF0707D0538199F800C0D5
:104B50002CF0020C89F800C00AE090F84670BFB152
:104B60004FF0020C012F18D080F8463080F81AC19F
:104B70000F0B67F34D310160802D2AD305F01F0123
:104B800058F821100C4201680CD041F004010BE0F0
:104B900080F8466080F81A31EAE780F846C080F86D
:104BA0001A61E5E721F0040101604C070DD44C05C2
:104BB0000BD5947AE40708D0538199F8005025F07A
:104BC000020589F80050C0F898308C0864F38A21F7
:104BD0000160917AC90717D1134991F8641001292E
:104BE00012D11249496C32290CDC0178490709D5E8
:104BF0000189090506D4D0F8981047F23054A14233
:104C000004D95681C0F89830BDE8F083491CC0F83B
:104C10009810F9E7E00500203C940008DA05002030
:104C2000580A0020A4020020B80C002048010020EF
:104C300010B5FCF797F80F48018821F002010180B8
:104C40000C49183109880C4A928E1144094A3432B1
:104C5000118008490C390A8842F001020A80011DBE
:104C60000A884FF6ED531A400A80018841F012017C
:104C7000018010BD0C04004050040020064841880B
:104C8000491C89B24180B1F57A7F04D38188491CDF
:104C900081800021418070473C0700200F4810B5FB
:104CA000016841F00101016041680D4A1140416015
:104CB00001680C4A11400160016821F48021016003
:104CC000416821F4FE0141604FF41F018160FFF74C
:104CD000C7FE05494FF00060086010BD001002409B
:104CE0000000FFF8FFFFF6FE08ED00E02DE9F041BF
:104CF0003149324D0888401C088028884FF0000454
:104D0000000629D5FCF7AEF92D4A2E48072317785F
:104D1000C8262D49012F22D02C4FB7F806C0BCF170
:104D2000000F3ED0B0F80CC04CF0080CA0F80CC03E
:104D3000B0F806C02CF4006CA0F806C0886820F01B
:104D400004008860FC801370CE8700204FF49661C9
:104D5000401C80B28842FBD32C80BDE8F0811C4F00
:104D600097F800C0BCF1010F0FD0BCF1020F11D0B9
:104D7000B0F806C04CF4006CA0F806C0886840F09B
:104D80000400886005203870DDE7B0F80CC04CF0F6
:104D9000080C03E0B0F80CC04CF0100CA0F80CC0EC
:104DA000F0E70C4F3C70C78847F40067C7808868FD
:104DB00040F004008860C6E73C070020102C01404A
:104DC0001B070020580A0020A402002064090020CC
:104DD0001C07002039070020704700002DE9F04330
:104DE0004FF08040018A21F001010182AC48007837
:104DF00000287CD1AB4FF87B002878D1AA48406CC2
:104E0000322874DCA9488068DFF8A4924104A94DD7
:104E1000B9F804004FF0000403D4401CA9F80400C2
:104E200028E1002874D02978012611B1012912D077
:104E300017E14946B0F5BE7FFAD92E70CC718C715E
:104E4000EC702C72287A0A18401CC0B214722872B6
:104E50000F28F7D305E1B9F802204946824201D96B
:104E6000EE7100E0EC7192488A7908300F2A15D271
:104E7000CB79082B0BD2C3F10708EB7912F800C0ED
:104E800003FA08F363441354CA79521CCA71CA79ED
:104E9000082A03D18A79521C8A71CC7199F80610BC
:104EA000C8460F2973D10D21FCF746F8A881010AE5
:104EB0006970C0B2A87088F8064098F816208A4237
:104EC00065D198F81510814261D198F80BC07A49E4
:104ED000032302227948BCF1000F10D0BCF1010F6E
:104EE00002D0BCF1020F14D080F86A2000E0CBE0C1
:104EF00091F800C02CF00C0C0CF1080C0FE080F8BD
:104F00006A6091F800C02CF00C0C0CF1040C06E067
:104F1000A9E080F86A3091F800C04CF00C0C81F8E0
:104F200000C098F80C10B6EB111F04D180F86E4049
:104F300087F846400EE0B2EB111F04D180F86E6096
:104F400087F8466006E0B3EB111F03D180F86E20AE
:104F500087F846200B0717D001F00F01012901D077
:104F6000022915D080F86C602C7198F80D102A7900
:104F700006FA02F30B406B71082A44D2DFE802F014
:104F80000B124319242F363D80F86C40ECE768E0A3
:104F900080F86C20E8E713B180F8704033E080F8C7
:104FA000706030E013B180F850602CE080F8504021
:104FB00029E023B180F8656087F8036123E080F879
:104FC000654087F803411EE023B187F8F54080F87B
:104FD0004D4018E087F8F56080F84D6013E013B19C
:104FE00080F868600FE080F868400CE013B180F84A
:104FF000666008E080F8664005E013B180F86760FD
:1050000001E080F86740521CD2B22A71082AAED360
:1050100098F80E102A4A8B0705D587F8F16080F8BA
:105020006460568104E087F8F14080F86440548160
:10503000C90702D080F8294001E080F8296098F87B
:10504000111000F86D1FC2781E48012A1ED001B34E
:10505000012921D04FF48051A0F876101A493C2044
:105060000870A9F80240A9F80440B9F80210491CD8
:10507000A9F80210B9F80210B1F5FA7F04D940F28C
:10508000F511A9F802102C70BDE8F08344F21C71F0
:10509000E2E74FF40051DFE741F25551DCE7000051
:1050A0001B070020A402002048010020001001403E
:1050B000A00C0020B4060020C8040020B80C00207A
:1050C000580A002030050020180700202DE9F05F65
:1050D000FDF726F98E4D2888A5F10406C0070AD0F1
:1050E000308820F008003080288820F009002880CF
:1050F00001F012FED9E02888DFF81892DFF8188254
:10510000864C80071AD5B9F8001041F00101A9F8C2
:105110000010B8F800008049143150300880288809
:105120004FF6F95108402880308840F00400308064
:10513000FEF71CFF84F83C00BDE8F09F2888784FFC
:105140004007288871D520F004002880FEF70EFF64
:1051500094F83C108142EFD1308820F00400308078
:10516000FDF7B6FA2078410605D594F84C1094F86E
:105170003B209142E0D03978400621F0020139709D
:1051800004D5FEF7D1F997F82F7004E094F83C00AD
:10519000FDF718F90746DFF880B140F68C2A0BF1CD
:1051A000180B062F47D294F83800B8423ED0384644
:1051B000FDF78CF82078C00716D094F83A0094F8E0
:1051C000391000F00302914206D0A17A00F00100EC
:1051D00001F00101884215D1FDF7E2F9FBF70EFE5F
:1051E000FDF70AFB384689E0FDF7DAF9FBF706FE22
:1051F000FDF702FB3846FDF7F3F9207840F0010097
:10520000207099E7288820F008002880206B81080A
:1052100001EBD000504515D2B8F800100844ABF8A7
:105220000000308840F0080003E00DE0308820F0F6
:105230000800308080E7B9F8001041F00101A9F8BA
:105240000010DFE75046E7E70007288831D520F057
:1052500008002880308820F008003080FEF786FEA5
:1052600084F83C00FDF734FA387820F002003870FA
:105270002078400604D5FEF757F997F82F5004E040
:1052800094F83C00FDF79EF80546062D08D294F8E8
:105290003800A842B5D0FDF783F9FBF7AFFD2AE04F
:1052A0002048C18841F04001C180BDE8F05FFDF7B2
:1052B00083BAC006288825D520F0100028803088C1
:1052C00020F01000308097F838000C2802D2401CE3
:1052D00087F83800387840F002003870FEF724F97B
:1052E00097F82F50787884F8390094F83800A8425D
:1052F00087D0FDF755F9FDF77FFA2846BDE8F05F46
:10530000FDF76EB94EF2BE110840288014E7000088
:105310001004004000040040240400404801002024
:1053200050040020580A00202DE9F04F514F85B05D
:10533000388820F0010038804E4800261030068062
:105340004D4CDFF838A14FF0010894F85C0042F6AC
:105350003029C10774D072B64948816941F400719F
:105360008161816941F4806181614FF40040FEF701
:1053700063FD444D00212846FBF79EFA0021284694
:10538000FBF790FADFF800B100215846FBF78AFAE4
:1053900000213E48FCF710F92846FBF7A9FB5846C8
:1053A000FBF7A6FB4FF46020CDE902068DF80560FF
:1053B00000968DF810808DF8048069462846FBF72A
:1053C00029FC01231A460F212846FBF774FC012112
:1053D0002846FBF767FA00204946401C80B2884205
:1053E000FBD328462E600121FBF7A4FC2868800728
:1053F000FCD524484C30006894F85C1021F0010181
:105400002144A1F85000FBF761FA62B6FDF798FF5E
:1054100047F69061AAF8001094F85C00401CC0B2F6
:1054200084F85C000C2822D212491431A1F80080C3
:10543000388840F00100388005B0BDE8F08FFFE704
:10544000134920F00100085A12490880114945F615
:105450005800083908800F4847F25801001F0180A2
:105460000C4920200C390880AAF80090D4E70320CA
:10547000A070E1E700080040500400202C08004024
:1054800000100240002401400028014008000240B2
:10549000F88F0008202C01400029018802D041F03B
:1054A000800101E021F080010180704710B50A8879
:1054B0004B88CC881A438B8823431A430B891A43A1
:1054C0004B8989891A430A43A0F8442010BD002162
:1054D000018041808180C18001814181818170474B
:1054E0000029818802D041F0010101E021F0010191
:1054F000818070470029018802D041F0010101E05C
:1055000021F0010101807047002930F8441F02D0CA
:1055100041F4004101E0C1F30E0101807047000039
:105520004B4910B5884202D10121C41486E0B0F184
:10553000804F09D0474988420DD101210220FEF752
:105540009DFC0021022064E001210846FEF796FC44
:10555000002101205DE04049884206D1012104205C
:10556000FEF78CFC0021042053E03C49884206D120
:1055700001210820FEF782FC0021082049E038497B
:10558000884206D101211020FEF778FC002110206E
:105590003FE03449884206D101212020FEF76EFC0D
:1055A0000021202035E03049884202D101214414F5
:1055B00044E02E49884202D10121CC043EE02C492E
:1055C000884202D101210C0538E02A49884202D1E3
:1055D00001214C0532E02849884206D101214020B2
:1055E000FEF74CFC0021402013E02449884206D1FC
:1055F00001218020FEF742FC0021802009E02049A3
:1056000088420AD1841501212046FEF737FC00218B
:105610002046BDE81040FEF731BC1A49884202D14D
:1056200001210C040AE01849884202D101214C04EE
:1056300004E0164988420AD101218C042046FEF775
:1056400035FC2046BDE810400021FEF72FBC10BD00
:10565000002C01400004004000080040000C004005
:10566000001000400014004000340140004C014094
:10567000005001400054014000180040001C004050
:10568000002000400040014000440140004801402B
:10569000002A828901D00A4300E08A438281704750
:1056A00030B5028C22F001020284028C8388048BC4
:1056B00022F0020224F073050C882C430D89154357
:1056C0004A882A43114DA8420BD0114DA84208D058
:1056D000104DA84205D0104DA84202D00F4DA8424F
:1056E0000DD122F008054A8923F440732A4322F0A1
:1056F00004058A882A438D891D43CB892B438380E7
:105700000483C9888186028430BD0000002C0140DA
:105710000034014000400140004401400048014085
:10572000028B22F008020A430283704770B5028C94
:1057300022F010020284028C8488038B0D8823F4EB
:10574000E6464FF6FF7303EA052535430E8922F03E
:10575000200203EA061616434A8803EA021232437D
:10576000104EB04202D0104EB04215D122F0800649
:105770004A8924F4406403EA0212324322F04006CC
:105780008A8803EA021232438E8903EA8606264398
:10579000CC8903EA8404344384800583C988018763
:1057A000028470BD002C014000340140028B4FF692
:1057B000FF7322F4006203EA012111430183704761
:1057C00070B5028C22F480720284028C8488838BF0
:1057D0000D8823F073031D4322F400730E894FF6E6
:1057E000FF7202EA06261E434B8802EA0323334374
:1057F000104EB04202D0104EB04215D123F40066D4
:105800004B8924F4405402EA0323334323F4806693
:105810008B8802EA032333438E8902EA0616264365
:10582000CC8902EA0414344384808583C988818743
:10583000038470BD002C014000340140828B22F0B3
:1058400008020A438283704770B5028C22F48052AA
:105850000284048C8288838B0D8823F4E6464FF6FD
:10586000FF7303EA0525354324F400560C8903EA47
:10587000043434434E8803EA06362643094CA042DA
:1058800002D0094CA04205D122F480448A8903EA5F
:105890008212224382808583C988A0F84010068442
:1058A00070BD0000002C014000340140828B4FF697
:1058B000FF7322F4006203EA0121114381837047E0
:1058C000018582827047828822F0700282808288FD
:1058D0000A4382807047A0F84010704730B50288B4
:1058E0001B4B1C4C98420DD0A0420BD0B0F1804F06
:1058F00008D0194DA84205D0184DA84202D0184D25
:10590000A84203D122F070054A882A43154DA842C7
:1059100006D0154DA84203D022F44075CA882A4308
:1059200002808A8882850A88028598420AD0A0422D
:1059300008D00E4A904205D00D4A904202D00D4A3E
:10594000904201D1097A01860121818230BD000097
:10595000002C0140003401400004004000080040D9
:10596000000C0040001000400014004000400140C6
:1059700000440140004801404FF6FF718180002142
:105980000180C1804180017270470029018802D0E6
:1059900041F0020101E021F002010180704700297D
:1059A000018802D041F0040101E021F004010180EE
:1059B00070470000224910B591F820000A6821497B
:1059C00000F01F0051F820001F490242086802D071
:1059D00040F4803001E020F4803008601B484FF034
:1059E0000003807941061A4827D41A4902880C8896
:1059F000A21A92B201240F2A0BD30A88028082686D
:105A0000002A00DA5242042A03DD134A1278022ADD
:105A100005D0427F012A06D00988418010BD447715
:105A2000C3770A88428042880988891A89B240F27D
:105A30001A629142F2D3C47710BD437710BD0000C3
:105A4000E00500203C940008A4020020580A002031
:105A5000800C0020240700201B0700202DE9F041C6
:105A60004D6800231E240F22854202DD0868BDE830
:105A7000F081D1F8F450854202DAD1F8F000F6E76F
:105A800001EBC2056D68854201DA134600E0144659
:105A9000E21852085D1CAA42F2D101EBC20351F890
:105AA00032505C68844202DAD3E9026701E053E9CC
:105AB0000267001BC11789053A1B41EA9021D317E1
:105AC0008005FAF72FFB721BA0FB024601FB026167
:105AD000D31700FB0310810241EA94502844C6E723
:105AE0002DE9F04FDFF8B8B16A48DFF8AC91DFF884
:105AF000ACA190F80EC0BBF91A70BBF91C60BBF9E1
:105B00001850BBF96C10BCF1070F48D2DFE80CF05D
:105B10008D041A30485E7600D9F800208284DAF8C5
:105B20000020C284828CC38CA7EB820212B2A6EB47
:105B300083034A431BB2594342F3CF2241F3CF239D
:105B4000D11870E0D9F800204284DAF80020C2842D
:105B5000428CA5EB820213B2C28C4B43A6EB8202AD
:105B600012B243F3CF24514341F3CF23E11814E0A1
:105B7000D9F80020C284DAF800204284C28C438C19
:105B8000A6EB820212B2A5EB83031CB24A43614327
:105B900042F3CF2341F3CF24191949420AB244E01A
:105BA000D9F800208284DAF800204284828C438C69
:105BB000A7EB820212B2A5EB83034A431BB25943FF
:105BC00042F3CF2241F3CF24111914E0D9F8002079
:105BD0004284DAF800208284428C838CA5EB820216
:105BE00012B2A7EB83034A431BB242F3CF245943BB
:105BF00041F3CF22A11849420BB216E0D9F8002098
:105C0000C284DAF800208284C28C838CA6EB8202E4
:105C100012B2A7EB83031CB24A4342F3CF23614382
:105C200041F3CF22991849420CB2BBF91E50594694
:105C300005F21E56A64201DACE8306E0A5F21E55F5
:105C4000A54201DDCD8300E0CC83B1F9204004F210
:105C50001E55954201DA0D8406E0A4F21E549442CA
:105C600001DD0C8400E00A84B1F9222002F21E5406
:105C70009C4202DAABF8224008E0A2F21E529A429D
:105C800002DDABF8222001E0ABF82230417B8173CA
:105C9000BDE8F08FA40200203C2401403C280140D4
:105CA000300500202DE9F04704466F48704D00266E
:105CB00002786E48022AB0F9301004D0082A7BD04E
:105CC000092A7AD0CBE0C27B022A02D1B0F8402068
:105CD00052B1A4F8421069810423B5F908101A469C
:105CE0000020FEF703FFB1E06249DFF88C81496ACA
:105CF0000F14E7808068410216D5B4F9020040F223
:105D0000DA21884248DD40F26A41884205DD00BF61
:105D10000823B4F942101A4660E0A0F2DA20FAF73C
:105D20007CFB0022554B68E0C0F3C001C0F30020AB
:105D3000DFF84C9181420CD1D8F8440040F2BA41CE
:105D400088426DDD40F66A118842E1DCA0F2BA407B
:105D50004FE04C480078C0060CD5D8F8440041F21A
:105D6000243188425CDD41F2D4718842D0DC00F6F7
:105D7000DC401EE04448DFF8149190F870100129CF
:105D80000BD090F86F00012807D041480178C9076F
:105D900046D04049098889B142E0B4F9020041F691
:105DA000DC6188423CDD42F23411884212DC00F5AD
:105DB0009270A0F500501CE04AE04EE0B0F91000EF
:105DC000B4F90210A0F59672914229DD00F59672A1
:105DD00091420BDDB4F9421020231A460020FEF751
:105DE00085FEA4F84200002817DB1BE0081A00F526
:105DF0009670FAF712FB00224B46FAF77AFA0E2257
:105E0000FAF7E6FAFAF740FB00B2C0F580407843B3
:105E10008013A4F84200002F04DCA4F8426001E0E3
:105E2000A4F84270B4F842001B4FE880D8F8441040
:105E30007964A7F84C0000F083FBB7F84E00688146
:105E400098F80A000028388F00D14042288106E0E7
:105E50001248B0F87C00688100E069812E8184F8E6
:105E60004060BDE8F08700001B070020A40200206E
:105E70006400002030050020480100200000794027
:105E800000C09240FC060020B80C002000C08240F8
:105E90004809002020000020F40800206C0A00209F
:105EA0002DE9F041B1F9025000232B24152285423F
:105EB00003DAB1F90000BDE8F081B1F9AE508542D6
:105EC00002DDB1F9AC00F6E701EB8205B5F902504D
:105ED000854201DD134600E01446E21852085D1CBD
:105EE000AA42F1D101EB8205B5F90230834206DA0C
:105EF00035F9026C35F9044C31F9221006E01E46E2
:105F000031F92240B5F90630B5F90410801B091BA0
:105F1000C5178911AD0345EA90458703A1FB070C1E
:105F2000CA1702FB07C201FB05219A1BD317FAF718
:105F3000F9F8000A40EA0160001900B2B0F5804F9C
:105F4000B9DB43F6FF70B6E770B5134C40F2244559
:105F50002946204600F03EF800281BD0204600F0DD
:105F6000C7F82946204600F01DF80C4C00212046B9
:105F7000FBF722FB2046FBF79DFBC0F164000849BC
:105F8000C0B20428087201D900F046F9BDE870409B
:105F9000FBF7D6BB70BD000000380140580002403E
:105FA0006C0600200A0A01219140C9430180704714
:105FB0000029818902D041F4005101E021F400510F
:105FC00081817047002A828A01D00A4300E08A4317
:105FD0008282704730B501F01F0201240025C1F311
:105FE000421304FA02F2012B0FD0022B0FD0838A46
:105FF0004FEA11210088134204FA01F400EA040078
:1060000001D000B10125284630BD8389F0E7038A1D
:10601000EEE710B5C1F3421301F01F040121A140C6
:10602000012B07D0022B07D01430002A026805D0BC
:106030000A4304E00C30F8E71030F6E78A430260C8
:1060400010BD000030B50446008A85B00D464CF600
:10605000FF710840E98801432182A1894EF6F310BF
:106060000140A8882A8910436A890A431043A08105
:10607000A08A4FF6FF410840A9890143A1826846E2
:10608000FDF720FF1948844201D1039800E00298EF
:10609000A189090400EBC00101EB0010296801D5BA
:1060A000490000E08900B0FBF1F06422B0FBF2F19E
:1060B00009010B096FF018056B4300EB8300A389FE
:1060C0001D044FF0320306D503EBC000B0FBF2F025
:1060D00000F0070005E003EB0010B0FBF2F000F069
:1060E0000F000843208105B030BD0000003801409A
:1060F0008088C0F308007047F8B501210920FDF73A
:10610000C9FE01218803FDF7C5FE10258DF8035057
:106110002020ADF800001A4E03248DF80240694695
:106120003046FCF745F816490C31086820F020008D
:10613000086018208DF803004020ADF800008DF8AD
:10614000024069463046FCF733F848208DF80300DA
:106150008020ADF8000069463046FCF729F88DF83C
:1061600003502801ADF800008DF802406946304622
:10617000FCF71EF801210420FCF76CF8F8BD0000C4
:10618000000C014030B585B0FFF7B6FF00244FF496
:10619000E1300090ADF808400C201D4DADF80440F2
:1061A000ADF80A00ADF80640ADF80C406946284647
:1061B000FFF748FF25208DF8100004208DF811000E
:1061C0008DF8124001208DF8130004A8FDF748FB5C
:1061D000012240F224412846FFF71BFF01212846F7
:1061E000FFF7E6FEFBF7D6FA012280212846FFF7EB
:1061F000E9FE012240212846FFF7E4FE01220221A8
:106200000448FBF76BFAFBF7C5FA05B030BD000098
:10621000003801404400024070B51D4D002428782C
:10622000432834D16878462831D1A878502807D03F
:10623000512805D0812803D0892801D0212826D1D2
:10624000144E7071E9787172A81C891CFAF7ACFEC3
:10625000B072717A294409793182884217D106F1E6
:106260000E00017841F0020101700B48016841F015
:1062700020010160317A0948002204E02B5D0355BA
:106280002A55641CE4B28C42F8D38078707170BDDA
:10629000B40700206C0600200C0C0140EA0B002023
:1062A00070B51D20FDF7BBFAFDF73EF91D20FDF787
:1062B000CCFA154890F82F10144D0623144C85F88D
:1062C000381090F83B1095F83B201143012A04D078
:1062D000022A07D0042A0AD010E0827A8A420DD01E
:1062E000007B09E0027D8A4208D0807D04E0827F45
:1062F0008A4203D090F82000884200D12370002009
:1063000085F8400070BD00005004002048010020C6
:106310001B0700200B4800214180A0F1B0018A89B1
:106320008280CB891A44C2800B8A1A4402814B8A2C
:106330001A444281898A1144818143F6FF71C181E7
:1063400070470000F8010020084940F61C72B1F9BE
:106350000C00904202DA00F59F7005E041F2E30282
:10636000904201DDA0F59F70C88170476400002055
:1063700038B51348C16941F00401C1611E208DF890
:10638000000002208DF801008DF8020001248DF834
:1063900003406846FDF764FA0A49842008800949E9
:1063A00047F690602C3108800020091F08800549BD
:1063B00014310C80091F0880081F048038BD0000BC
:1063C000001002400008004030B420491E4A4578C1
:1063D0008B7A114692F83B4091F83910AC4218D1B3
:1063E0004BB10379994202D04379994201D1407966
:1063F0001AE0807909E08379994202D0C479A142F8
:1064000002D182F82F3011E0407982F82F0030BCA1
:106410007047C578AC42FAD16BB1C379994202D0CA
:10642000037A994205D1007A82F82F0030BCFEF73A
:10643000FFBB407AE9E7437A9942E2D00479A1426E
:10644000DFD0007AE1E7000050040020480100207E
:10645000FEE700002DE9F0470446007F012868D1DF
:106460003548E1880288511A89B2072916D3008875
:10647000E080B4F9000044F2DD414843401346F6A1
:10648000D96148438013A060401000B2A0814FF052
:106490008051B1FBF0F0F9F7BBFF2061B4F90C605B
:1064A00096B1B4F902104DF6B05048430014A082E2
:1064B000B4F904704DF6B05207FB02F24FEA2245E0
:1064C000E58204D4024603E00020E08330E042424B
:1064D00012B22283002D01DB2B4600E06B421BB27F
:1064E000DFF85890638398464FF4804AB24208DA46
:1064F000F9F785FF2169F9F758FEF9F7ACFF80132A
:1065000004E0002901DA484600E05046E083B04547
:1065100009DA2846F9F773FF2169F9F746FEF9F71A
:106520009AFF801304E0002F01DA484600E050464D
:106530002084BDE8F08700002407002000C0FFFF92
:1065400010B52248234C01782148022905D1C17B8E
:10655000022902D1B0F8401029B1008EA4F84E00F3
:106560000020208710BD90F846101A48B0F844006B
:1065700000B239B318490978C1F3810101291BD050
:1065800002291CD0154900BFFBF76AFC1149A4F889
:10659000400080B2483101F091FAB4F94C00B4F9EE
:1065A0004A2041425143891324F8381FB4F910108E
:1065B00048438013E08210BD0849D839E4E7074911
:1065C0006C39E1E705496C31DEE700001B0700206C
:1065D000A4020020F4080020C8040020708D0008E8
:1065E0000348002180F82A10C1830187704700000A
:1065F000F408002010B504000B462D4AC3F100003A
:1066000028D56442002B12DAA04207DA214600F0B6
:106610002DFA32F81000C0F5404041E00146204616
:1066200000F024FA32F8100000F5004038E0A342F0
:1066300008DA2146184600F019FA32F8100000F581
:1066400040402DE0204600F011FA32F81000C0F56D
:10665000803025E0002B12DAA04207DA214600F054
:1066600005FA32F8100000F5804019E00146204696
:1066700000F0FCF932F81000C0F5004010E0A34231
:1066800008DA2146184600F0F1F932F81000C0F59A
:10669000804005E053B1204600F0E8F932F81000E0
:1066A000B0F5004F01DDA0F5803010BD002010BD19
:1066B0000490000840438013494300EBA1300022BE
:1066C0000302002B14DDB3F5001F01DC802001E084
:1066D0004FF4005093FBF0F1014401EBD1714910EC
:1066E000814206D0521CD2B20846062AF2D300E0FC
:1066F0000021C80000B2704702E008C8121F08C19C
:10670000002AFAD170477047002001E001C1121F32
:10671000002AFBD1704700002DE9F047A74CA8489C
:1067200021880288511A89B20F297DD30088A4F1EB
:106730003C052080288F08B1401E288795F800C0AE
:10674000A04ACCF3810001281DD0022820D0D18B93
:106750009D4E9A48DFF87492F388407E0027B1F589
:10676000926F1CD8142818D37820607643F010005C
:10677000F08040F26660A8812CF001002870D77389
:1067800089F8007018E0D08B00EB4000C00302E0F5
:10679000D08B8F494843010CDAE7401C04E0B1F587
:1067A000DB6F09D310B1401E607605E023F01000C6
:1067B000F0804CF001002870B5F90200B5F91430F2
:1067C0004143C3EBC303C1F38F31C3F3D10303EBE5
:1067D000510109B2A9829046D28B4FF080535043A9
:1067E000B5F91620C0F38F30C2EBC202C2F3D1025A
:1067F00002EB500000B2E882AA6A42431213EA6236
:1068000093FBF2F22A63734A1080A2680A44A260E2
:10681000E1680144E160207C401CC0B2207407287C
:1068200002D942F3CF0000E0C5E02883C910698394
:10683000E760A76041F6C8012774884204DD298B10
:10684000654AB2FBF1F1E981C117890341EA904140
:10685000800342F69B420023F9F764FCA884574862
:106860005E49A0F13C002A78B0F906005FEA827C1C
:1068700000FB01F14FEA2143C2F3810115D5012943
:1068800007D002290BD04FF2685141430914A1806F
:1068900011E049F68C4148430014A08020E04CF6FA
:1068A000183141430914A18026E001290ED00229A4
:1068B00018D0A0806B844A4948430014A4F81E00F5
:1068C000FBF7EEF847480088C0B143E04AF65C3178
:1068D00041430914A1804BF62C21484300146884DD
:1068E000E383EDE74DF2AC5141430914A1804EF230
:1068F0007C414143091469843B49DDE795F8200058
:1069000000BB88F80F7089F80070B5F91A00A0F57F
:106910000C519F39B1F56E7F18D8617FF42912D9D7
:106920003249E8802E4AA1F8460050430014A8805E
:10693000A1F84400FF2085F8200081F828002C49A8
:106940003C20087006E0491C617703E0607F08B1D5
:10695000401E6077B5F91A10B4F91E0081420EDDB1
:10696000A07E7D2809D9F08840F00800F0802148F9
:10697000017821F0020101700EE0401C06E0A0F257
:106980003D10814208DAA07E10B1401EA07603E0DF
:10699000F08820F00800F080B5F91810606908440C
:1069A0006061217E491CC9B221761F2903D940119B
:1069B000A88367612776BDE8F08700000405002002
:1069C00024070020A4020020580A00201B070020F2
:1069D000303301000C0A002074E8260BCC0E0100B5
:1069E0004885010026070020D0450100B80C002092
:1069F00018070020DA050020024941F68B30886232
:106A000070470000C804002070B5164C0625207899
:106A1000062825D2DFE800F003080E141A211248D8
:106A2000FAF700FB012016E00F48801DFAF7FAFA8A
:106A3000022010E00C480C30FAF7F4FA03200AE0C8
:106A400009481230FAF7EEFA042004E0064818303C
:106A5000FAF7E8FA0520207070BDFAF703FB2570FD
:106A6000257070BD1C070020488E0008090A05D05B
:106A7000B0FBF1F0FF2800D9FF20704700207047DD
:106A8000D0E90021C368521A5A4301EBA231816058
:106A900041607047B0F90020B0F90210B0F906303B
:106AA000521A5A4301EBA2318180418070470000A5
:106AB00030B5494B188849490A8A801A85B2484836
:106AC000484A0F2D047801F150001DD31D880D8216
:106AD000117A090713D5022C01D0434912E0434D26
:106AE000B0F90210B5F90050A94205DC02DA01F153
:106AF000020108E0458007E0A1F1020103E0022C59
:106B000002D13B4909884180B0F840101D88691ABC
:106B100089B29C2949D31988A0F84010916A0023B2
:106B2000B1F5804F31DB3349896CB1F5405F2CDD25
:106B3000314940F26665B1F91010A94212DD43F601
:106B40009915A94202DB40F2333108E040F23335B7
:106B5000A1F26661694343F2333591FBF5F1A0F888
:106B6000441001E0A0F844302449B2F806510978F5
:106B7000C1F381012DB100BFB0F8441001F21E51E4
:106B80001CE092F84620022A10D0A0F84430022CD3
:106B900001D0A0F84430B0F95C10B0F9443001F1F4
:106BA00014029A420DDAA0F85C2030BD012901D010
:106BB0000229E1D1B0F8441001F23331A0F84410B9
:106BC000E5E703F11402914203DD1439A0F85C10EB
:106BD00030BDA0F85C3030BD240700201400002038
:106BE0001B070020A4020020C6040020C4040020CB
:106BF000C00400204801002030050020C804002007
:106C00002DE9FC4101210220FDF72CF90121192079
:106C1000FDF740F901213C48FBF71CFB4027ADF88C
:106C2000007003248DF802400420384D8DF80300D5
:106C300069462846FBF7BCFAE001ADF800008DF884
:106C400002401C208DF8030069462846FBF7B0FA85
:106C50004FF4E0712846FBF732FBA815ADF80000B1
:106C60008DF8024010208DF8030069462848FBF794
:106C70009FFA4FF4A060FCF725FE1D208DF804005C
:106C800001268DF8056000258DF806508DF8076007
:106C900001A8FCF7E5FD1F498C2008801D494FF62F
:106CA000FA702C3108806E20091F088019481430B2
:106CB0000680184808300780164920310D80154A93
:106CC000D020121D1080134A45F2F30018321080B4
:106CD0000A1F45F2500010800E4A4FF6FF703832FE
:106CE0001080121D1080121D108041F21B100880B0
:106CF00000F012F8FBF760FD064810300580001F19
:106D00000480BDE8FC810000000C1A000010014066
:106D1000000C01400004004070B51D20FCF774FD1C
:106D20002A4D40212846FBF7C1FA840080212846DD
:106D3000FBF7BCFA44EA4004A9152846FBF7B6FA6B
:106D40000443E0B2224C84F83C00FBF73BFB0546D1
:106D5000052805D91F48C18841F04001C18001E0E4
:106D600084F838501C48007A000703D594F838009E
:106D70001A490D5C4FF6FA702063E062A06260620F
:106D80002062E061A0611648606300206064A06436
:106D900084F83F0084F84000FBF7C2FAA07AFF288D
:106DA00011D0022084F83D000E4800882066284655
:106DB000FBF764FF207820F001002070BDE87040F0
:106DC0001D20FCF737BD0120ECE70000001001405A
:106DD00048010020580A0020A40200200099000861
:106DE000DCFF0500240400402DE9F0434E484F49E4
:106DF00002880B889A1A92B20F2A69D309880180F7
:106E00004B49098B027D00EB42029180017D491CB8
:106E1000C9B2017508295BD3002404752246017D9F
:106E200000EB4103491CB3F90430C9B202EB630221
:106E300012B201750829F2D33E4904753E4B4A80CF
:106E400044800E789D895FEAC67C40F638694FF031
:106E5000030714D0A2F22B5C42F6E858C44520D3B5
:106E6000A1F1020C26F00204ACF8002047750C706A
:106E700040F22B54A24211DA45F004021EE046F023
:106E800001060E704A4507DD45F001029A8126F0A1
:106E900002020A70477519E0447517E045F00202D6
:106EA0000CE04A450CDA8775427D12B1521E4275DC
:106EB0000CE046F002020A7025F007029A8105E014
:106EC000B30703D5837D2BB15B1E83754088888013
:106ED000BDE8F08342F6AA239A4222DAB1F90430DF
:106EE0002BB941F2CD05AA4201DA4480EEE7134CFA
:106EF000920302EB843241F67244B2FBF4F214B214
:106F000040F2333502464480AC4200DA5580B2F993
:106F10000240E41A04F5A374B4F5237FD6D8438065
:106F2000D4E74FF48043FAE7EC0A0020240700205E
:106F3000A4020020DA050020580A0020C8F1FFFF53
:106F40002DE9F0416D4CDFF8B8E14FF0000594F801
:106F50003410C80706D094F938104B42002958DD88
:106F60000E4657E0674884F83750A4F84250664A06
:106F700090F8380084F840001586CEF80450CEF81A
:106F80000850624E40F26663CEF80C50A4F87C3094
:106F900036F810005E4E768830444FF6FF7606EAEB
:106FA000800024F8300B4FF0806044F8040CA320DC
:106FB000208460845810A084E38440F699102085D2
:106FC000580060854FF48050A08541F23330E08551
:106FD00041F26660208641F69910608641F6CC4009
:106FE000A0864FF40050E08642F23330208742F210
:106FF0006660608742F69910A08742F6CC40E08731
:1070000082F89D5041F00100207184F84450BDE8A1
:10701000F0811E4694F937004242002801DD074600
:1070200000E01746F61B012E0BD0002800DB0246BD
:107030005FFA82F684F8380094F84F00012805D0F2
:1070400041E0002900DA1946CEB2F3E794F939306D
:107050005942002B01DB184600E0084694F93A201B
:10706000C7B25042002A01DB944600E08446BC458A
:1070700008DD002A00DA0246D7B2002B00DA0B4600
:10708000D8B207E0002B00DA0B46DFB2002A00DBA3
:107090001046C0B204EB4000B0F9501004EB4700BA
:1070A00030F9502F11444910018084F84F5084F872
:1070B0003E5084F83D5084F83C5084F83B5084F8AE
:1070C0003A5084F8395004EB46007546B0F9500048
:1070D00024F8420FBEF80410C82309B26422FDF759
:1070E00005FD6860E968401AA9680844A860B5F918
:1070F00000104843C013E860608788E76C0A0020EE
:10710000C805002048010020A402002012990008B0
:1071100064000020F0B4544890F83410C90776D0C9
:10712000524990F84030002291F838108B426FD0CD
:107130004F4CA0F872204F4DE65C04468E4294F905
:10714000374002D0EE5C8E420FD1641C64B280F8EE
:107150003740EB5C8B4202D1641C80F8374090F9D9
:1071600037300F2B1BDD0F2317E0434DEE5C434DF3
:107170008E4202D0EE5C8E4211D1641E64B280F861
:107180003740EB5C8B4202D1641E80F8374090F9A7
:1071900037406FF00E039C4201DA80F83730324BF3
:1071A00090F83F50393390F83740EC5490F83F3026
:1071B0005B1CDBB280F83F30062B01D380F83F2008
:1071C00090F9394090F93B309C420ED190F93D4006
:1071D000A3420AD190F93A4090F93C309C4204D144
:1071E00090F93E40A34200D1012280F84F201F4A6F
:1071F00080F8401090F937501378214A012D0DDDA9
:1072000014465E07A46804D544F0080403E028E0AF
:1072100015E024F00804946080F83510B5F1FF3FC4
:107220000ADA5B07936802D523F0080301E043F014
:107230000803936080F83510F0BCFBF771B890F844
:107240004F1001290DD1B0F8721043F60953491CB3
:1072500089B2A0F87210994203D9A0F8722080F880
:107260004F20F0BC704700006C0A0020480100204D
:10727000F4980008FA980008069900080C9900088C
:10728000A402002010B5D0E900210369114481FB5C
:1072900003318C0244EA93514260D0E9022382FB1D
:1072A0000332940244EA93521144816010BD0000FD
:1072B00030B52049204AB1F86A301088C01A80B22F
:1072C0000F2836D31088A1F86A001C4D00204FF01B
:1072D00000432A5C940903D00124B4EB921F24D10B
:1072E000D20622D0164A52F820201268134C1234CB
:1072F00034F81040224201EB000494F9722008D0C7
:107300000A2A04DB0A6823FA00F4224308E0521C2C
:1073100009E012F10A0F05DC0A6823FA00F4A2431F
:107320000A6002E0521E84F87220401CC0B211288C
:10733000CFD330BDE00500202407002008940008CA
:10734000089500082DE9F00779497A480A890388E9
:107350009A1A92B2082A74D300880881A1F12C00ED
:1073600042890AB1521E4281734A92F82820802A2B
:1073700067D302F03F020A70C2890AB1521EC2816D
:10738000B1F90620902A0CDB8A46FF2A09D08146F3
:10739000C089002855D1694800230078092805D004
:1073A00005E0BDE8F007624800F09EB90823644A92
:1073B00092F8EA500DB143F004036248817AC9079C
:1073C00001D043F00203D2F808C05FEA0C5101D5A6
:1073D00043F00103176800215B4EFC0302D596F8C9
:1073E000654004B18021C4885FEA446801D541F05A
:1073F00040015FEA845801D541F020015FEAC4787A
:1074000001D041F01001007A400701D541F0080198
:107410004E480078C00701D041F00401A00601D514
:1074200041F001010020012D00D1082096F8705094
:1074300085B992F84620022A04D0012A05D03AB133
:1074400008E072E040F0030004E040F0020001E0D8
:1074500040F001007A0701D440F02000CCF3C002D4
:107460000025CCF3002C624502D13A0700D4042554
:1074700096F86F20012A01D145F00105344A002712
:10748000BC4612783E46C2F38102012A04D0022A89
:1074900004D0032A04D004E0022602E0042600E01F
:1074A00010262C4A64060ED5214C1C342478240660
:1074B00009D51478640606D4274A40F6CC44926D68
:1074C0006243140C05E0B2F8AE2040F69914624312
:1074D000940B4FF008088AF80A804FF061088AF888
:1074E0000B808AF80C308AF80D108AF80E008AF8A2
:1074F0000F508AF81070270A4B4083F06901414011
:1075000069408AF8117079408AF812406140524609
:107510008AF813C071408AF8146051754FF4C8712D
:10752000A9F80E10FF20AAF80600BDE8F007704782
:10753000E006002024070020E00500201B070020B3
:10754000A4020020580A0020B80C0020480900209E
:10755000C804002048010020180800205148816913
:1075600041F0FC0181614FF4A060FCF7ABF9FBF73F
:10757000B1F9FCF70BFBF9F713FBFCF701F9FDF789
:10758000BBF9FFF73DFBFCF741F8FFF7C5FBFBF745
:1075900013F9454D45494FF40050A5F81601886789
:1075A000FEF7F0FD00214FF4FA5340F2EE220020E6
:1075B000401C80B29842FBD3491C89B29142F6D359
:1075C0003B48002680F87260F9F780F9F9F72EFE43
:1075D000FCF70CFBF9F7F4FCFEF7CAFE1022354964
:1075E0003548F8F7D0FD01F0F7F9344C354FE08815
:1075F00020F04000E0803248017821F02001017045
:10760000FA20F8814FF49670E887FFF7F5F92E49D4
:107610002E48FCF768FA2E48FCF78AFA2D48416A92
:1076200088472D48416B8847FEF7DAFF2B48FAF769
:1076300033FA2B494220C8802A49C8603E71E0884D
:10764000E0812089208260896082FAF729FDFAF7BB
:107650008BFCFFF761F801F05FF9FFF7C5FB00F065
:10766000FBF9FFF725FE01F01BF8FEF7A3F9FAF787
:10767000E7FAFBF721FBFFF71BFAFCF7F1FCFAF73F
:1076800043FFFAF775FF00F07DF8FFF75BFE134844
:10769000FAF7CAF800F06CFAFDF772F9FAF732FA65
:1076A000CDE7000000100240A4020020640000208A
:1076B00030050020B80C002020060020580A0020C9
:1076C0004801002018070020C4080020940800206A
:1076D0000804002038000020E4000020D809002021
:1076E000440700203C040020F0B523490278B0F99B
:1076F000064000231F4E31F81210FF2C18D0B0F9AD
:1077000004701E4DBC4231DA00EBE40704F00704BC
:10771000BF7AA7408478FFB23CB190F801C0ACF1C9
:10772000010C64451FDA3C061DD455F822200DE0FB
:1077300056F82220116012498A79521CD2B28A71FD
:10774000022A02D38370C3808B71F0BD11608178EF
:10775000491CC9B2817042789142F6D38370C188C6
:10776000491CC180F0BD56F82220EFE755F82220D1
:107770001160F4E7E89500081A9400089095000855
:10778000B4060020F0B561486149B0F86C200B8860
:107790009A1A92B29C2A7BD30988A0F86C105D4992
:1077A0005D4F91F82A1001F0070297F84610022A5F
:1077B00000D1491E594C80F83E104FF00203E28878
:1077C0004FF00001550401D5012236E0A489E506F9
:1077D00001D5062231E0250701D508222DE0550606
:1077E00003D44F4D2D78AD0601D5042225E01505B3
:1077F00001D5072221E0150601D50A221DE09506D4
:1078000001D50C2219E0150701D50B2215E055070B
:1078100001D4D50501D510220FE0D50601D50522EA
:107820000BE0650703D4A50701D4E40702D080F874
:107830006E3007E0920403D5032280F86E2001E049
:1078400080F86E10374A384C92F820E0324A251FF3
:10785000D2F808C02D4AB2F87060721C92B2BEF124
:10786000000F0DD02CF4000CC7F808C090F86E7013
:10787000B7B11E2F1AD090F86F200AB325E007E0A9
:107880004CF40006BE60A0F870200A2A01D22360E2
:10789000F0BD142A01D22B60F0BDA0F87010F0BD2D
:1078A0002B60A0F8701080F86F10F0BD642E04D229
:1078B000A0F87020322AEED3E9E7A0F87010EAE7CA
:1078C0007F1C80F86F70A0F8701090F86F20012A6C
:1078D00010D0002AE9D0B0F87060761CB6B2A0F8DB
:1078E00070601E2ED7D323603C2EDED9521E80F846
:1078F0006F20D2E7B0F87020521C92B2A0F870202E
:107900002360C82AD1D980F86F10C6E7E0050020AF
:1079100024070020B80C0020A4020020580A0020F0
:1079200048010020C8040020141C0140F0B5424862
:10793000B0F84810491C89B2A0F8481002297AD33F
:107940003E490024A0F848400A783D4B042A57D00D
:107950004FF48041082A0BD0A0F10C02B2F90020AC
:107960008A4200DA1146B3F980208A4200DA1146D1
:10797000344A92698A4200DA11B2418282881D8AB1
:10798000C2EB8502304D12B22D78C5F381062A4D27
:1079900042F291767243B5F9765092126A4312130D
:1079A000C26086681546C6EBC60642F3D102F602EF
:1079B00002EBA6328260C66C1644C664B0F8507002
:1079C0007F1CBFB2A0F85070B7F5806F04D3B61219
:1079D0000682A0F85040C464891A1C4EC26A7243E1
:1079E00040F255564E4302EB4602466A324442622A
:1079F000B3F93030B2EB034F06DD1A04426206E001
:107A00001349B1F90410B3E7002A00DA4462C162F5
:107A1000104990F83D2091F838108A420BD080F838
:107A20003D10B0F84210A0F84410B0F84010A0F893
:107A30004210A0F84050F0BD300500201B07002088
:107A4000A4020020500C0020C8040020C3F5FFFF52
:107A50006C0C00204801002015481649B0F85A2047
:107A60000B889A1A92B20F2A20D30988A0F85A10CC
:107A7000B0F9001041F6515251438913A0F86C102F
:107A80000D494FF480420B78A0F10C01022B06D176
:107A9000B1F90030934202DA1B1D0B8000E00A802E
:107AA0000021A0F8601020F85C1F428070470000A1
:107AB00030050020240700201B0700204FF6FF722E
:107AC00002EA800210F4404315480ED0B3F5804F0F
:107AD00014D0B3F5004F4FEA122216D0C2F58073CE
:107AE00030F813305B424B8005E0120A30F8123058
:107AF0004B80C2F5807230F812000FE0120AC2F516
:107B0000807330F813304B8005E030F81230C2F546
:107B100080725B424B8030F8120040420880704710
:107B200004920008104A518A908AD28A163846393F
:107B3000A2F1110200D54942002A00DA5242114452
:107B4000002800DA40420844084943F6284300B2BE
:107B5000B1F936205A43921340F2D733584302EB1F
:107B6000A030C88670470000A40200203005002025
:107B7000F0B5904990480A8903889A1A92B23E2A31
:107B80001ED30088088101F138004FF4FA63428A5D
:107B90009A4202D2521C428200E04382874A92F803
:107BA0002220802A0CD302F03F020A70B1F906208D
:107BB000402A06DBFF2A04D0C2883AB1521EC28096
:107BC000F0BDBDE8F0407B48FFF78EBD428A9A4287
:107BD000F6D307784FF0010E3A074FF0FF055BD55B
:107BE000847A40F2DC52630708D444F004038372C1
:107BF000C28081F80BE081F80AE04CE04378072B63
:107C000005D0032B03D0052B01D0062B07D1660628
:107C100005D444F040038372C280052239E0654AEE
:107C20005FEA437C02F138024FF42076127A0DD5D8
:107C30005FEAC26C0AD45FEA446C07D442F01002D7
:107C400002723A0628D4C680192222E0DF0709D042
:107C5000970707D4670605D442F002020272C68075
:107C6000042216E09F0709D5170707D4670605D435
:107C700042F008020272C68003220AE01B070BD5FD
:107C8000530709D4630607D442F004020272C68087
:107C90000B22CA728A72CD80494AB2F92230B2F9F7
:107CA0001A7003F23D140022A74200DB0276414E17
:107CB000444C06F13806A479B6895FEAC46C06F133
:107CC00001064FF4C874B6B213D58681B6F57A7F33
:107CD00005D9017A21F0800101728281F0BD037A19
:107CE0001E06FBD4828143F080020272C480112000
:107CF00035E09F4216DA037E052B13D28681B6F556
:107D0000487F04D98281027A22F040020272027A0C
:107D10005606E3D45B1C037642F040020272C48034
:107D200002201CE0284B1C89C4F3C006C4F30027C2
:107D300040F2EE24BE4216D11E78360713D4427E9E
:107D4000012ACBD1428BB2F5167F02D2521C42835C
:107D5000F0BD827A42F002028272C4800F20C872A3
:107D60008872CD80F0BD93F80D714FF40046012F5D
:107D700018D1164F41F6583C7F6C674512DD83F8E9
:107D80000CE1134B1E60C38AA34202D25B1CC38268
:107D9000F0BD4FF4FA73C3801C23CB728B72CD807D
:107DA000C282F0BDC2820A4883F80C21001F06601F
:107DB000F0BD0000C406002024070020E0050020DC
:107DC000C8040020580A0020A40200204801002016
:107DD000140801402DE9F05FFE48FF49DFF8FCA3DD
:107DE000007E0A1D131D012850465AD030F85A4F04
:107DF0000C8041881180BAF85E001880FDF770FE93
:107E0000F74DF84C49F2CD32B5F91E006083B5F953
:107E1000201043F6CC4C00EB410151430914A183DF
:107E2000B4F92230B4F9206001FB03F200FB062212
:107E300042F38F326282B4F9167007FB0CF7BF135E
:107E400040F2333C714302FB0CF200FB131007EBD2
:107E5000A232E28240F38F30A082B4F91810E24FD0
:107E6000C1EBC10141F3D10101EBE000DF4E208302
:107E7000786C3060316930468847DD493089488008
:107E80000846FDF70FFFDFF86CB301264FF000093D
:107E90009BF8000008280CD0618F218204287DD037
:107EA0001AE030F8604F0C8041881180BAF8640005
:107EB000A3E7D14890F93710491C02296FD890F8F0
:107EC000741019B1B4F85A00208205E0618F218244
:107ED000A4F85A1080F87460B4F91410B4F90A00C8
:107EE000C64AF9F7DDFAE062BAF91611884204DDF4
:107EF000C248E162027C91408162BA48DFF800E347
:107F0000503847F2A30802784EF24611002A79D081
:107F1000012A78D080F800909BF8000004287FD0D8
:107F2000B64AB4F91210B4F90800303AF9F7B8FAC1
:107F300043F26661A062884200DBA162A346254647
:107F4000A06AAE4C443C2060E86A60602046103570
:107F5000FCF760F8A34928883C39FFF7AFFDDFF84C
:107F60008482A8F15008D8F81410C8F87010B5F938
:107F70001010A068B5F9123000FB01F7E268584311
:107F800002FB137444F38F3702FB0100AF8740F309
:107F90008F34EC879B4D6F80AC8001E03DE03AE090
:107FA0002846FEF757FA287F08F11805012878D0EF
:107FB000604241104DF6B350474369803A142A801D
:107FC0004046A8F804408B18C380891AA8F8081006
:107FD0008AF80C90B8F904305446002B00DD267363
:107FE000B8F90600002802DD217B891C2173B8F94D
:107FF0000820002A02DD217B091D2173217B07292E
:108000007ED202E011E036E00AE0DFE801F0807C99
:10801000947A907E9200608F56E7686A0014E0625E
:10802000B87AE8B37848A06288E7B5F91E204244E0
:108030008A420AD8B5F9202042448A4205D8B5F9C7
:10804000222042448A427FF667AFA0F80290B7F838
:10805000AE204946B2F5C87F01D8467006E0B2F5B9
:10806000487F01D8022200E0032242708AF80F10F4
:108070008BF8001027E080F80090B5F91EC04A4642
:10808000C4448C4509D8B5F920C0C4448C4504D8F3
:10809000B5F9225045448D42D5D9B7F8AE1001E06C
:1080A0001AE01CE0B1F5C87F01D8467006E0B1F5D2
:1080B000487F01D8022100E00321417042808AF804
:1080C0000F208BF80020BEF8061041F40061AEF8D6
:1080D0000610F9F73BFF1FE74FF4AF70A3E74948DD
:1080E0004DF6B352B0F92030594249106980B0F9C9
:1080F0001E00504302142A804046A8F8043062E76C
:1081000005E0667303E0022100E0032161739BF840
:1081100000103E4E01293E4F617BDA460DD0072903
:1081200078D2DFE801F077FEFDFCFBFAF9000421CC
:10813000ECE70521EAE70621E8E70729F0D2DFE8C6
:1081400001F069042F7FA4D8F10001461846FBF71F
:10815000B1FC2860B5F9020040F681514843811313
:108160006980B5F9000040F68152504380132880A1
:108170000A18A2F68152B8F80E305242C3EB6202DE
:1081800012B2A8F80C20002A01DCA8F80C90B8F86C
:108190000C20A4F85E201144A4F85C10084479E196
:1081A000404201B2504200B2FBF784FC2860B5F9AE
:1081B000020040F68151484380136880B5F90010F1
:1081C00040F68152514389134218A2F68152298008
:1081D000524220E0D8090020342C0140A4020020A3
:1081E0003005002064000020480100203C040020ED
:1081F000F80300201B0700206C0A0020C4080020A0
:10820000580A00200C0A0020A2FEFFFF00240140B3
:1082100000280140DDE0B8F80E30C3EB620212B274
:10822000A8F80C20002A01DCA8F80C90B8F80C2063
:1082300058E13046F8F712FD01231A460721BDE048
:1082400019461046FBF736FC2860B5F9020040F6E7
:108250008151484380136880B5F9001040F681527F
:108260005143891329804218A2F68152B8F80E3082
:108270005242C3EB620212B2A8F80C20002A01DCC1
:10828000A8F80C90B8F80C2059E15942404209B2C4
:1082900000B2FBF70FFC2860B5F9020040F68151EF
:1082A000484381136980B5F9000040F6815250437C
:1082B000801328800A18A2F68152B8F80E30524274
:1082C000C3EB620212B2A8F80C20002A01DCA8F865
:1082D0000C90B8F80C20A4F85A201144A4F85C10B3
:1082E000084462E13046F8F7B9FC01231A4605213B
:1082F00064E01146FBF7DEFB2860B5F9020040F6AA
:108300008151484381136980B5F9000040F68152DC
:1083100050438013288006E080E154E125E1F6E037
:10832000C6E099E017E00A18A2F68152B8F80E30BC
:108330005242C3EB620212B2A8F80C20002A01DC00
:10834000A8F80C90B8F80C20A4F85C201144A4F80C
:108350005A10084454E1504201B2584200B2FBF7AF
:10836000A9FB2860B5F9020040F68151484381130A
:108370006980B5F9000040F681525043801328808F
:108380000A18A2F68152B8F80E305242C3EB6202CC
:1083900012B2A8F80C20002A01DCA8F80C90B8F85A
:1083A0000C20A4F85C201144A4F85E10084455E1A8
:1083B0003046F8F753FC01231A4606213846F8F7F1
:1083C0004DFC01213046F8F7BFFB01213846F8F794
:1083D000BBFBB04EBAF8080055463080BAF80A0028
:1083E0007080BAF81000B0803046F9F769FAB4F836
:1083F0005A00F1880844A4F86000B4F85C003189A0
:108400000844A4F86200B4F85E0071890844A4F836
:108410006400317EA048012978D034F85A1F0180C9
:1084200061884180A18881809B49028808310A8047
:1084300042884A80808888809748896A08308847BF
:1084400095F83E0000287DD0F8F70CFE15F83E0F99
:10845000401E2870BDE8F09F01461846FBF72AFB36
:108460002860B5F9020040F68151484380136880C6
:10847000B5F9001040F68152514389134218A2F613
:108480008152524252082980A4F85E201044A4F878
:108490005C000844A4F85A0000213046F8F754FB69
:1084A00000213846F8F750FB01231A460621C0E6A2
:1084B000404201B2504200B2FBF7FCFA2860B5F925
:1084C000020040F68151484380136880B5F90010DE
:1084D00040F68152514389134218A2F6815252420A
:1084E00029805208A4F85E201044A4F85A000844D9
:1084F000A4F85C0000213046F8F726FB002138463E
:10850000F8F722FB01231A46052192E6B4E019464A
:108510001046FBF7CFFA2860B5F9020040F681510A
:10852000484380136880B5F9001040F681525143EA
:1085300089134218A2F68152524229805208A4F8A7
:108540005A2000E09BE01044A4F85E000844A4F820
:108550005C0000213046F8F7F7FA00213846F8F7BA
:10856000F3FA01231A460721BCE65942404209B2F8
:1085700000B2FBF79FFA2860B5F9020040F681517E
:10858000484380136880B5F9001040F6815251438A
:1085900089134218A2F68152524252082980A4F847
:1085A0005A201044A4F85C000844A4F85E0000219E
:1085B0003046F8F7C9FA00213846F8F7C5FA012322
:1085C0001A4606218EE61146FBF774FA2860B5F9C3
:1085D000020040F68151484380136880B5F90010CD
:1085E00040F68152514389134218A2F681525242F9
:1085F00052082980A4F85C201044A4F85A000844CA
:10860000A4F85E0000213046F8F79EFA00213846B3
:10861000F8F79AFA01231A460521C9E6504201B239
:10862000584200B2FBF746FA2860B5F9020040F65E
:108630008151484380136880B5F9001040F681529B
:10864000514389134218A2F681525242520829809E
:10865000A4F85C201044A4F85E000844A4F85A0072
:1086600000213046F8F770FA00213846F8F76CFA26
:1086700001231A4607219BE634F8601FCFE607481E
:108680000088A0F5D04168393FF4E4AEBDE8F05F62
:10869000F9F7AABBD809002030000020182C0140AF
:1086A0002DE9F041904C9148B4F85A100288511AC3
:1086B00089B20F296FD30088A4F85A008C4800882B
:1086C000DFF83082C0074FF000054FF0010741D0BE
:1086D000874AD4E90C1024321388B1EB530F02D22D
:1086E0001288511A08444FF4F371884200D20846A8
:1086F0008149B1FBF0F0616CC1F3510108440646B9
:108700006064F7F78AFE00227C4BF7F7F2FD4FF02A
:1087100040427B4BF7F7EDFD0E22F7F759FEF7F7D6
:10872000B3FEA4F8A40094F86500401CC0B284F81D
:108730006500082834D36C4898F84620001F037859
:108740009A4201D0027045806E4A13786E4A23B176
:10875000458021E06564A56458E0D8F89410A1F53F
:10876000FA618E4211DD616D8B1C9E4205DDB0F910
:1087700002100A290DDA491C06E08E4205DAB0F92A
:108780000210002908DD491E4180B0F902000A28C4
:1087900002DB177001E0A2E01570666584F8655091
:1087A0005A484FF4A5420178C1F38101012949D00B
:1087B00002294AD044F687712181A4F8A020B0F99B
:1087C000243089B24B439B13A4F89C30B0F90E00BF
:1087D00000237043B0FBF1F0A16CC0F3D100C1EBFA
:1087E000C101C90200EB9130A064F017810341EA96
:1087F0009641B003F7F796FCB4F8A210C1EBC101A3
:10880000C902C00800EB9130A4F8A200616CA06E10
:108810000844A06694F86C20521CD2B284F86C20F4
:10882000082A05D3C008A4F86E0084F86C50A56629
:108830003748384EC3885A0633D498F80F20022A96
:1088400006D02CE043F20451B6E744F24621B3E7E8
:10885000B26840F69916B24221DD94F8382094F8B7
:108860008660B2420CD084F8862094F83D2002F055
:108870000106C2F34002964202D1A4F8825004E0FD
:10888000B4F88220B2F5966F05D2B4F88200401C8D
:10889000A4F8820005E043F08002C28001E0A4F861
:1088A0008250114894F83F30B0300C2B01D2C5747F
:1088B00000E0C774174A0F4C41F2482692F83C205A
:1088C000B4F8824041F2504C0C2B0AD3B14208DB81
:1088D000012A06D0614502DD002C00D18774BDE875
:1088E000F0818574FBE70000480100202407002088
:1088F00000040040A40200204564BD0100209C400B
:10890000133B3340F6030020F7030020C804002087
:10891000580A00203005002070B5284C28482188CE
:108920000288511A89B23E2947D300882080254801
:10893000808B254D80022860696928468847234935
:10894000A868FDF78BF822496060CB885A072ED4BF
:108950000022B0F1F05F0FD9E089B0F5FA7F08D9B5
:1089600043F00400C8801B48017821F00201017027
:108970001CE0401CE0811AE0B0F1D25F0CD94FF44A
:10898000F031A1EB10308003C910B0FBF1F0206191
:1089900000280CDA22610AE0B0F1C85F03D94FF475
:1089A0008040206103E023F00400C880E281D4E924
:1089B0000401884200DB0846A06170BD500C002015
:1089C00024070020A40200208C060020FC97000849
:1089D000580A0020DA05002005494FF4804048611C
:1089E000086188610348C18821F48271C1807047A1
:1089F000500C0020580A00202DE9F041384C394E27
:108A0000394F207841F23331C2074FF000050CD0C6
:108A1000A28962B394F90700002800DA4042C0B28C
:108A2000032829D240F2AE702AE0A570E5732F4AE0
:108A3000E571A58192F83830237220F00800A180FA
:108A400040F0020020703D867560B560F560916C65
:108A5000490005D041F68461A18140F010002070EA
:108A6000C0B240F0010020706574BDE8F0816581FE
:108A700020F01000207015E0042803D240F65100C9
:108A800060810FE0052802D240F69910F8E740F621
:108A9000CC42062803D3072801D3082801D26281DB
:108AA00000E0618197F89D0098B9B088102301B269
:108AB000B4F90A003622FCF719F87060F168401A20
:108AC000B1680844B060B6F900104843C013F060C4
:108AD0003886388E10B10120A070C6E7A570C4E7B3
:108AE0006C0C0020A4060020A402002048010020F5
:108AF0002DE9F041554C2678F0077CD05448217A76
:108B0000544D90F8380081427BD0534A2346DFF819
:108B10004CC1575C93F90E2093F90730874203D07C
:108B20001CF80170874213D146F002065B1C2670C8
:108B30005BB2E3711CF80110814201D15B1CE3714F
:108B400094F90710062901DD0621E171521C1CE091
:108B5000434F17F801C0434F844503D017F801C0B5
:108B6000844513D126F002065B1E26705BB2E371CA
:108B7000795C814201D15B1EE37194F907306FF09B
:108B800005018B4200DAE171521EA273207294F942
:108B900007108A1C042A02D941F68462A2812C4A59
:108BA000012912780ADD2B4B56079B6802D543F04A
:108BB000080301E023F00803AB606070B1F1FF3FF0
:108BC00009DA5107A96802D521F0080101E041F056
:108BD0000801A9606070F9F7A3FBA078012810D103
:108BE00021488068A3280CDA94F90700022803DDE5
:108BF0000220E07105E01EE06FF00101884200DA1A
:108C0000E171A089002630B1401E0004000CA08153
:108C100001D1E671A673E87B04280CD0B5F93010B9
:108C2000512341220020FBF761FF2886002802D152
:108C3000E07B10B1A670BDE8F0810C4806700C48CE
:108C40000670207820F001002070F4E76C0C002002
:108C500048010020A4020020F4980008FA980008B7
:108C6000069900080C9900083005002038070020FC
:108C70001B070020743F713D9B3BED396238F43691
:108C8000A13565343F332A32273133304C2F722ED1
:108C9000A32DDF2C242C722B000000361C0700387B
:108CA000AA0A003AAA0A003CCC0C003ECC0C0040B8
:108CB000380E0042380E0044380E0046380E004888
:108CC000380E004AC711004CC711004EC7110050A2
:108CD000C7110052C7110054C7110056C7110058E0
:108CE000C711005AC711005CC711005EC7110060B0
:108CF000C7110062C7110064C7110066C711006880
:108D0000C711006A00000036220200388E03003AC4
:108D1000B005003CD207003EF4090040160C0042AA
:108D2000380E00445B100046C71100483313004A58
:108D30009F14004C9F14004E0B16005077170052E2
:108D40007717005477170056771700587717005A8F
:108D50007717005C7717005E77170060771700625F
:108D60007717006477170066771700687717006A2F
:108D700000000036FA04003C6606003ED2070040C0
:108D80003E090042F4090044AA0A0046600B00486C
:108D9000160C004ACC0C004C820D004E380E0050D0
:108DA000EE0E0052A40F00545B1000561111005833
:108DB000C711005A7D12005C3313005EE913006096
:108DC0009F140062551500640B160066C1160068FA
:108DD0007717006A2D18006CE318006E000000344D
:108DE00000000036000000380000003A0000003C9F
:108DF0000000003E0000004000000042000000446F
:108E000000000046000000480000004A0000004C3E
:108E10000000004E0000005000000052000000540E
:108E200000000056000000580000005A0000005CDE
:108E30000000005E000000600000006200000064AE
:108E40000000006600000068441458585870111162
:108E50005858587041115858487011144858587053
:108E60001411584858703313005695130054B61314
:108E700000525A140050FD14004EA115004C451626
:108E8000004A761600486C17004672180044BA195A
:108E90000042741B0040911D003EB420003C9F2204
:108EA000003AE1220038532300368B240034812518
:108EB00000322B2700302028002E5829002CB02A01
:108EC000002A9B2C0028D22D00267C2F002426313E
:108ED000002202330020FD34001E5C37001CCC3C15
:108EE000001A873E0018BE3F0016004000140040E4
:108EF0000012004000100040000E0040000C004036
:108F0000000A004000080040000600400004004045
:108F100000020040000000200072002000700020CD
:108F2000006E0020006C0020006A00200068002015
:108F30000066002000640020006200200060002025
:108F4000005E0020005C0020005A00200058002035
:108F50000056002000540020005200200050002045
:108F6000004E0020004CA320004AA32000484721C7
:108F70000046EB210044EB2100428F2200408F226B
:108F8000003E7A24003C7A24003A662600385128B4
:108F900000343D2A0030702D002CA33000287A3494
:108FA000002451380020CC3C001C00400018004038
:108FB0000014004000100040000C00400008004079
:108FC0000004004000000000010203040500050049
:108FD000010203040104000305020000F001000087
:108FE00036010000F8000000BA0000007C0000001C
:108FF0007C0000007C000000411414111114441185
:10900000141441110000290052007B00A400CC0080
:10901000F5001E01470170019901C201EA01130226
:109020003C0265028E02B602DF02080330035903D8
:109030008203AA03D303FB0324044C0475049D0498
:10904000C504EE0416053E0567058F05B705DF0567
:1090500007062F0657067F06A706CE06F6061E074A
:1090600046076D079507BC07E4070B083208590847
:109070008108A808CF08F6081D0944096A09910962
:10908000B809DE09050A2B0A520A780A9E0AC40AA0
:10909000EA0A100B360B5C0B820BA80BCD0BF30B03
:1090A000180C3E0C630C880CAD0CD20CF70C1C0D8C
:1090B000410D650D8A0DAF0DD30DF70D1C0E400E41
:1090C000640E880EAC0ECF0EF30E170F3A0F5E0F24
:1090D000810FA40FC70FEA0F0D1030105310751039
:1090E0009810BA10DD10FF1021114311651187117E
:1090F000A911CA11EC110D122E12501271129212F6
:10910000B312D412F41215133613561376139613A2
:10911000B713D713F6131614361456147514941483
:10912000B414D314F214111530154E156D158C1599
:10913000AA15C815E7150516231641165F167C16E5
:109140009A16B716D516F2160F172C174917661769
:109150008317A017BC17D917F51711182E184A181E
:10916000661881189D18B918D418F0180B1926190B
:1091700042195D1978199219AD19C819E219FD192A
:10918000171A311A4C1A661A801A991AB31ACD1A7C
:10919000E61A001B191B331B4C1B651B7E1B971B00
:1091A000AF1BC81BE11BF91B121C2A1C421C5A1CBA
:1091B000721C8A1CA21CBA1CD21CE91C011D181DA1
:1091C000301D471D5E1D751D8C1DA31DBA1DD01DB4
:1091D000E71DFD1D141E2A1E401E571E6D1E831EF8
:1091E000981EAE1EC41EDA1EEF1E051F1A1F2F1F6B
:1091F000451F5A1F6F1F841F991FAE1FC21FD71F05
:10920000EC1F002000006400C9002D019201F7014D
:109210005B02C00224038903ED035204B6041A055D
:109220007F05E3054706AB060F077307D7073B0823
:109230009F0802096609C9092D0A900AF30A560B0C
:10924000B90B1C0C7F0CE20C440DA60D090E6B0E25
:10925000CD0E2F0F900FF20F5310B4101511761181
:10926000D71138129812F8125813B813181477142B
:10927000D61435159415F3155116B0160E176B1735
:10928000C91726188318E0183D199919F519511AAC
:10929000AD1A081B631BBE1B181C731CCD1C261D9E
:1092A000801DD91D321E8A1EE31E3B1F921FEA1F1E
:1092B00041209820EE2044219A21EF214522992235
:1092C000EE2242239623E9233C248F24E2243425F2
:1092D0008525D72528267826C82618276827B72762
:1092E00006285428A228EF283D298929D629222A90
:1092F0006D2AB82A032B4D2B972BE12B2A2C722C8D
:10930000BB2C022D4A2D912DD72D1D2E632EA82E5C
:10931000EC2E302F742FB82FFA2F3D307F30C03015
:10932000013141318131C13100323F327D32BA32B7
:10933000F73234337033AC33E73322345C34953452
:10934000CE3407353F357735AE35E4351A365036ED
:109350008536B936ED36203753378637B737E93794
:10936000193849387938A838D738053932395F394A
:109370008B39B739E2390D3A373A603A893AB23A1D
:10938000DA3A013B283B4E3B733B983BBD3BE03B0D
:10939000043C263C483C6A3C8B3CAB3CCB3CEA3C26
:1093A000093D273D443D613D7D3D993DB43DCE3D68
:1093B000E83D013E1A3E323E493E603E763E8C3EDE
:1093C000A13EB53EC93EDC3EEF3E013F123F233F8A
:1093D000333F433F513F603F6E3F7B3F873F933F6B
:1093E0009E3FA93FB33FBC3FC53FCD3FD53FDC3F8C
:1093F000E23FE83FED3FF13FF53FF93FFB3FFD3FE7
:10940000FF3FFF3FFF3F0000E7382C35002020EFF3
:109410002037202333202620210000800200040072
:10942000080010000002000400080400000200040C
:1094300000080010002000400080040000000080B0
:1094400000000040000000200000001000000008A4
:109450000000000400000002000000010000800085
:109460000000400000002000000010000000080084
:109470000000040000000200000001000080000065
:1094800000080140000C0140000C0140000C0140AC
:10949000000C0140000C0140000C0140000C014098
:1094A0000010014000100140001001400010014078
:1094B0000010014000100140001001400010014068
:1094C0000014014004080140040C0140040C014058
:1094D000040C0140040C0140040C0140040C014048
:1094E000040C01400410014004100140041001402C
:1094F0000410014004100140041001400410014018
:10950000041001400414014008080140080C014007
:10951000080C0140080C0140080C0140080C0140F7
:10952000080C0140080C01400810014008100140DF
:1095300008100140081001400810014008100140C7
:109540000810014008100140081401400C080140B7
:109550000C0C01400C0C01400C0C01400C0C0140A7
:109560000C0C01400C0C01400C0C01400C10014093
:109570000C1001400C1001400C1001400C10014077
:109580000C1001400C1001400C1001400C14014063
:1095900010080140100C0140100C0140100C01405B
:1095A000100C0140100C0140100C0140100C014047
:1095B0001010014010100140101001401010014027
:1095C0001010014010100140101001401010014017
:1095D0001014014000000000000000000000000026
:1095E000000000000000000014080140140C0140BD
:1095F000140C0140140C0140140C0140140C0140E7
:10960000140C0140140C01401410014014100140CE
:1096100014100140141001401410014014100140B6
:109620001410014014100140141401400000000007
:10963000000000000000000000000000000000002A
:10964000FFFFFF0F0FFFFFFFFFF0FFFFFF0FFFFF09
:10965000FFFFF0FF0FFFFFFFFFF0FFFFFF0FFFFF18
:10966000FFF0FFFF0FFFFFFFFFF0FFFFFF0FFFFF08
:10967000FFFFF0FFFFFF0FFFFFFFFFF0FFFFFF0FF8
:10968000FFF0FFFF00000040400000000004000069
:109690000040000000000400400000000004000042
:1096A0000040000000040000400000000004000032
:1096B0000040000000000400000040000000000422
:1096C0000000004000040000000000808000000056
:1096D000000800000080000000000800800000007A
:1096E000000800000080000000080000800000006A
:1096F000000800000080000000000800000080005A
:1097000000000008000000800008000000000020A9
:109710002000000000020000002000000000020005
:1097200020000000000200000020000000020000F5
:1097300020000000000200000020000000000200E5
:1097400000002000000000020000002000020000D5
:1097500000000060600000000006000000600000E3
:10976000000006006000000000060000006000002D
:10977000000600006000000000060000006000001D
:10978000000006000000600000000006000000600D
:109790000006000000800200040008001000000223
:1097A000000400080400000200040008001000206B
:1097B0000040008004000000FF7FFFFFFDFFFFFF6F
:1097C000FBFFFFFFF7FFFFFFEFFFFFFFFFFDFFFFC7
:1097D000FFFBFFFFFFF7FFFFFBFFFFFFFFFDFFFFAB
:1097E000FFFBFFFFFFF7FFFFFFEFFFFFFFDFFFFFC5
:1097F000FFBFFFFFFF7FFFFFFBFFFFFF0000401FDA
:109800007A1903000000001E897603000000C01CC6
:109810003BDF03000000801BD15704000000401A0A
:109820009FE00400000000199E7B05000000C017A7
:10983000E42C0600000080160DF80600000040151C
:1098400093DE07000000001408E608000000C012C4
:10985000B1110A000000801101650B0000004010EA
:10986000E6E30C000000000F46940E000000C00D5F
:10987000467710000000800CB08F12000000400BF3
:10988000D2DE14000000000A5E6317000000C0086A
:10989000601A1A000000800726FC1C000000400629
:1098A00000002000000000057A1923000000C0031A
:1098B000D5392600000080025851290000004001DF
:1098C000764F2C000000000046252F000000C0FE4F
:1098D0002AC63100000080FDA1283400000000FBF2
:1098E0004B1F3800000080F829053B00000000F6FF
:1098F000EFFE3C0001020304050002030405000121
:10990000030405000102050001020304040500012F
:10991000020355050010AA1A55250030AA3A000086
:10992000AA0A55150020AA2A5535FF3F4C99000870
:109930000000002050070000E4060008489A0008D4
:1099400050070020E00900000867000845020406EF
:10995000082D010203040405480607080913652BB6
:109960001B087904211355152A4006190801A7136D
:109970006F3D1B0895041A8F040125170206040584
:109980000103148020FF8BAA0A02019C15AA0A5524
:109990001500085920AA2A5535FF3F07290301055C
:1099A00004060203127C1573FFFF04FF808001018F
:1099B00029025F6402130A13816A12081201100C53
:1099C0000504060203010103070505280B01020334
:1099D000040206070303040C3D0706040509191FCA
:1099E000191904310506064BAA1A024B381E0269E2
:1099F00010312E40FD3969260211042F405F020C00
:109A000026405B262ACD55155515123902017F03D4
:109A100016D0071AFF01013B0261AA0C12080108C7
:109A2000A8147F993F2340331385720A1608DC91EE
:109A3000220312100A17401C12600A16901B014DD7
:089A400013956A020008000002
:020000040800F2
:10FC00004A46545A594D46312D4E3330202020203B
:10FC1000050406020301AA0AAA0AAA0AAA0AAA0A4B
:10FC2000AA0ADE3F00100000FF0131000201664613
:10FC300000400040513800400040004000400101B9
:10FC400000400040FF387B257B257B25FF003333B8
:10FC50000201401F00016626B81E6626FFFFFFFF57
:10FC6000FFFF01010100010001000300000200008C
:04FC70000000AA5591
:04000005080000ED02
:00000001FF
